:10000000026CCC026DED00000000000269F60000F9
:10001000000000026E14000000000002281400001E
:10002000000000023EC80000000000026B04000057
:1000300074A21200C4E81200FFE91200FF12013698
:100040002274A21200C4E81200FFE71200FF09D5D3
:1000500082F81201362274A21200C4E81200FF7462
:10006000A31200C412011FF709D58204120136221F
:10007000C296D297000000C29780E974A21200C411
:10008000E81200FF1200882274A31200C412011F9C
:10009000F91201362274A27A08C296000000C297B3
:1000A000335005D2960200AAC296D297000000C231
:1000B00097DAEDD29600D297000000309604C297EE
:1000C000C322D3227A08D296D29700000000000003
:1000D00000000000000000000000C296000000C206
:1000E00097335005D2960200EBC296D297000000DB
:1000F000C297DAEDD29600D297000000C297227A1A
:1001000008335005D29602010BC296D29700000028
:10011000C297DAEDD29600D297000000C297227AF9
:1001200008D296C29700000000D297C3309601B360
:1001300033DAF0C29722C296000000D29700000086
:10014000D29622787D76000876007881E6543FF6D4
:100150007800797DC082758207120041D082120535
:10016000DB227802797FC082758205120056D08228
:10017000227883E603C4540775F018A4C0E07881A0
:10018000E6C4540375F00AA4F5F0E6540F25F0D048
:10019000F025F075F03CA4C0F0C0E07880E6C454CF
:1001A0000775F00AA4F5F0E6540F25F0D0F025F01D
:1001B000F5F0D0E03400C5F02250523330322076D2
:1001C00065722E3132352E32204864773A4720341A
:1001D000303030752031342D31312D3034203132F2
:1001E0003A34392020284329526F676572205370B2
:1001F0002E4A2E207777772E726F6765722E706C7D
:100200002C2074656C2F666178202B3438203535AE
:100210002032373230313332202843296A502D7052
:100220006C2C204D6F6E61204C6973612043452C0E
:100230002049534F393030312C2031737420436CB6
:10024000617373D320202052204520532045205431
:10025000D25052333032204C434420763132352E46
:1002600032004350523A20004C6F633A20004C4F0A
:10027000433A2000D22020202020202020202020AF
:100280002020202020D200454E545259202020000A
:1002900045584954202020200044555459204558A1
:1002A000495400494E5445524E414C0020202020D4
:1002B000200020D1466C6173682043524320457270
:1002C000726F722000D32053657276696365204F88
:1002D0004E00D32053657276696365204F46460011
:1002E000D2204D4153544552204944203D20203FC7
:1002F0002000D32020202055205320452052D220FA
:100300002050726F6772616D6D696E6700D2202038
:100310002020202020202020202020202020D2D576
:1003200001055245473A200000D3D5021044206F02
:100330002077206E206C206F206120642000D12067
:1003400020202020202020202020202020202020AD
:10035000D1D5030C50617373776F72643F203A20DC
:1003600000D2D50410204163636573732064656E09
:10037000696564202000D2D5051020416363657350
:1003800073206772616E7465642000D1D5041020FB
:100390004163636573732064656E6965642020D270
:1003A000D50610204E6F204475616C20456E747226
:1003B00079202000D3D509104475616C20456E74F6
:1003C0007279204D6F64652000D1D50A0A20202063
:1003D0004572726F722023002020202000D1D50C9E
:1003E0001020202041504220526573657420202047
:1003F0002000D2D50E104C696D6974206578636554
:1004000065646564202000D50F0C4E4F524D414C61
:1004100020202020202000D1D5041020204143435B
:100420004553532044454E59202020D2D51010204A
:100430004150422056696F6C6174696F6E202000D4
:10044000D1D50D10202020204964656E74204F4BBB
:1004500020202020D2D51010204150422056696F14
:100460006C6174696F6E202000D2D51110204E6F20
:10047000206F6E6520696E73696465202000D1D598
:1004800012102020456E746572204944203D203FA3
:10049000202000D1D5041020204143434553532050
:1004A00044454E59202020D2D506102020496E7098
:1004B000757420426C6F636B73202000D1D50410DB
:1004C00020204143434553532044454E592020208A
:1004D000D2D507102020434C4F534544204D4F4464
:1004E0004520202000D1D50410202041434345530E
:1004F000532044454E59202020D2D508104F757402
:10050000206F662074696D65207A6F6E6500D1D5A5
:10051000041020204143434553532044454E592065
:100520002020D2D50B10204F464620636F6E6469A1
:1005300074696F6E202000D1D513102020535749C5
:100540005443482044454E59202020D2D508104F0E
:100550007574206F662074696D65207A6F6E650012
:10056000D1D5131020205357495443482044454EB9
:1005700059202020D2D51610202020496E70757485
:100580002064656E7920202000D1D5041020204100
:1005900043434553532044454E59202020D2D5147F
:1005A0001020202020505245414C41524D20202007
:1005B0002000D1D50410202041434345535320440B
:1005C000454E59202020D2D5151020204C696D6948
:1005D00074202D2066756C6C202000C28E53890F0C
:1005E000438910758BD6758D97C28FD28E308FFD53
:1005F000C28E22C28E53890F438910758BEB758D85
:10060000CBC28FD28E308FFDC28E22C28E53890F05
:10061000438910E58AC4242BF58B758DEBC28FD2EC
:100620008E308FFDC28E22F9C3137004A24F801842
:1006300014C0E0030303540F247DF8D0E0540704F2
:10064000F5F0E213D5F0FCE992E02275F00612070E
:100650000222C2A075F006120702D2A02212065290
:1006600012064B12065212064B12065212064B127B
:10067000065212064B12065275F01812070222C2D9
:10068000A075F04B120702D2A022755204123C0A48
:10069000C2A075F0C8120702D2A022755205123C02
:1006A0000A12067F75F01E12070212067F2275528B
:1006B00007123C0A12066922755206123C0A1206FB
:1006C0006F2212065D12065D22755207123C0A75F2
:1006D0005206123C0A12066F12066F12066F2212A1
:1006E000066F12066322C2A1C26412065275F0128E
:1006F000120702D2A1C2642212065275F01212072A
:1007000002221205DB201A07C0F0122F69D0F0D5A3
:10071000F0F0227004A24FB322C0E014120722D0DE
:10072000E022C0E0030303540F28F8D0E0C0E054F7
:100730000704F5F0E213D5F0FCD0E022E575B40033
:1007400003020817B40717C2AC12060B12060BD22D
:10075000991208D7C25BD2B6126B0F020814B4010B
:1007600017C2AC12060B12060BD29912151DC25BF2
:10077000D2B6126B0F020814B40317C2AC12060BE8
:1007800012060BD2991215A2C25BD2B6126B0F02DF
:100790000814B40217C2AC12060B12060BD299123F
:1007A000143EC25BD2B6126B0F020814B40417C217
:1007B000AC12060B12060BD299121480C25BD2B691
:1007C000126B0F020814B40517C2AC12060B120606
:1007D0000BD299120840C25BD2B6126B0F020814FA
:1007E000B40617C2AC12060B12060BD2991215EA08
:1007F000C25BD2B6126B0F020814B40917C2AC1256
:10080000060B12060BD29912671CC25BD2B6126B92
:100810000F020814757500E56F6013B401051232FC
:100820007C8008B4020512328B8000756F00122F95
:100830006930460B20A808306105C2611232B82227
:10084000C2B612016275380074031250B9E51E1267
:1008500050B9E51F1250B974571250B97882E62387
:100860002354031250B97883E630E402240A540F6B
:100870001250B97882E6C4540375F00AA4F5F0E684
:10088000540F25F01250B97881E6C4540375F00A6C
:10089000A4F5F0E6540F25F01250B97880E6C45460
:1008A0000775F00AA4F5F0E6540F25F01250B97858
:1008B0007FE6C4540775F00AA4F5F0E6540F25F05E
:1008C0001250B97883E603C454071250B9E53812C0
:1008D00050B93099FDD32212694CC2B675380074F4
:1008E000031250B9E51E1250B9E51F1250B97450E9
:1008F0001250B9747D1250B9900000E536600F9027
:1009000003E81460099007D0146003900BB87E7D53
:100910007F0875F000C0F0126947B40203D380016C
:10092000C3D0E033F5F0A3DFEC1250B9DEE2E538D6
:100930001250B93099FD22C0F075F0DCD5F005B247
:10094000841264A1C0F0120B81D0F030E7EED0F039
:1009500022AAF0120937E5336530F5F0E534653148
:1009600045F0600C120AA8853033853134120937FE
:10097000120B46120937120B6E120937120AB58A8A
:10098000F022AAF0120937E5336530F5F0E5346559
:100990003145F0600C120AA88530338531341209D4
:1009A00037120B32120937120B6E120937120AB5C1
:1009B0008AF02279207530017531037532E090009C
:1009C000D8120937120AA8120937120B06790075D6
:1009D00030017531047532009000F8120937120A9F
:1009E000A8120937120B0679E075300175310575CB
:1009F00032009001F8120937120AA8120937120BB7
:100A00000685303385313422AAF0120937E5336583
:100A100030F5F0E534653145F0600C120AA88530F8
:100A200033853134120937120AEE8AF022AAF01205
:100A30000937E5336530F5F0E534653145F0600C94
:100A4000120AA8853033853134120937120AD68A42
:100A5000F022C0F075F00833C297929000D297D57B
:100A6000F0F5D0F022C0F075F008C297D29700A23E
:100A70009133D5F0F5D0F022D292D297D290D29184
:100A8000D29322E53133E5303322C3E5313322E519
:100A90003222120A52120A83120A52120A8A120AC5
:100AA00052120A8F120A5222120A78C293745312F7
:100AB0000A92D29322120A78C2937458120A92D2DE
:100AC0009322120A78C2937454120A92E4120A52C0
:100AD000120A65D29322120A78C2937454120A92AF
:100AE000E4120A52120A65F608D9F9D29322120AC0
:100AF00078C2937454120A92E4120A52120A65F2EE
:100B000008D9F9D29322120A78C2937454120A9225
:100B1000E4120A52120A65F0A3D9F9D29322120AFA
:100B200078C0E0C2937484120A92D0E0120A52D2C2
:100B30009322120A78C2937484120A92E6120A521D
:100B400008D9F9D29322120A78C2937484120A92B5
:100B5000E2120A5208D9F9D29322120A78C2937487
:100B600084120A92E0120A52A3D9F9D29322120AED
:100B700078C2937483120A92D2931205DB1205DBBA
:100B800022C2937457120A52120A65D29322D2904B
:100B9000D291D297D292D293B28475F0021205DB31
:100BA000D5F0FAC292B28475F0021205DBD5F0FAE4
:100BB000D292B284227530017531DB753200120990
:100BC00037120E507533FF7534FF22AE83AD82901D
:100BD000DB007F207404F9747DF875300185833162
:100BE000858232120A2D787DE66E702508E66D70DA
:100BF0002008E6601AB4FF028013167404F9747DAD
:100C0000F8753001858331858232120982C322D37F
:100C100022A3A3A3A3DFBD80F490DB007F20740494
:100C2000F9747DF8753001858331858232120A2D81
:100C3000787DE66E700908E66D700408E6FC22A374
:100C4000A3A3A3DF0A7CFF2290DB007F207BFF743D
:100C500004F9747DF8753001858331858232120A7A
:100C60002D787DE66E702C08E66D702708ECB4FFD9
:100C70000D787D76FF0876FF0876FF0874FFF6741E
:100C800004F9747DF875300185833185823212094B
:100C900082C322BBFF10787DE6B4FF0A08E6B4FFEA
:100CA00005C374209FFBA3A3A3A3DFA3BBFF02D3B1
:100CB00022EB232354FC2400F5827583DB500205CC
:100CC00083787DEEF608EDF608ECF608E4F6740499
:100CD000F9747DF87530018583318582321209827D
:100CE000C32275830075F08E7530028583317532AD
:100CF00000C0F0C083120937120E50D0830583D094
:100D0000F0D5F0E475830075F0DA75300385833132
:100D1000753200C0F0C083120937120E50D083051F
:100D200083D0F0D5F0E47533FF7534FF227583006E
:100D300075820075F08EC0F0C082C0837530028568
:100D40008331753200120937120AA8D083D082C0CD
:100D500082C08375300085823175320012093712E6
:100D60000B6ED083D08205830582D0F0D5F0C77595
:100D7000830075820075F0DAC0F0C082C0837530E0
:100D800003858331753200120937120AA8D083D047
:100D900082C082C0837530018582317532001209AC
:100DA00037120B6ED083D08205830582D0F0D5F048
:100DB000C77533FF7534FF2275830075820075F0A7
:100DC0008EC0F0C082C083753000858331753200DB
:100DD000120937120AA8D083D082C082C08375302E
:100DE00002858231753200120937120B6ED083D022
:100DF0008205830582D0F0D5F0C775830075820027
:100E000075F0DAC0F0C082C083753001858331751A
:100E10003200120937120AA8D083D082C082C08360
:100E2000753003858231753200120937120B6ED08E
:100E300083D08205830582D0F0D5F0C77533FF7566
:100E400034FF22120A78C2937450120A92D293226B
:100E5000120A78C2937481120A92D29322120A78EB
:100E6000C2937484120A92E8120A52D9FAD29322D7
:100E7000AAF0120937E5336530F5F0E53465314500
:100E8000F0600C120AA8853033853134120937120C
:100E90000E5D120937120B6E8AF022120A78C29385
:100EA0007454120A92E4120A52E4C0E0120A65D0A5
:100EB000F025F0D9F5D29322758300758202800661
:100EC000758300758200E475F08D858230858331ED
:100ED000753200C082C083C0F0C0E0120937120A28
:100EE000A81209377900120E9BD0F025F0D0F0D06F
:100EF00083D0820583D5F0D28582308583317532E7
:100F000000C0E0120937120AA81209377920120E20
:100F10009BD0F025F07533FF7534FF227583007583
:100F200082038006758300758201E475F0DA85829C
:100F300030858331753200C082C083C0F0C0E012BA
:100F40000937120AA81209377900120E9BD0F02532
:100F5000F0D0F0D083D0820583D5F0D27533FF7501
:100F600034FF05E02275830075F00075300085833D
:100F700031753200C0F0C083120937120E50D08391
:100F80000583D0F0D5F0E47533FF7534FF75830029
:100F900075F0DA753001858331753200C0F0C08399
:100FA000120937120E50D0830583D0F0D5F0E475C6
:100FB00033FF7534FF22120675754CFA3001FA754D
:100FC000F0051205DBD5F0FA754CFA2001FA222261
:100FD00022222222300D597882E6540FC0E0E6C466
:100FE000540375F00AA4D0F025F0FD7883E630E4D0
:100FF00002240A540FFE901A007F3C7404F9740016
:10100000F8753001858331858232120A087800E252
:101010006D701708E26E701208E2C42354E0F5F018
:101020007883E6541F45F0F68006A3A3A3A3DFCB85
:1010300022120162120FD4120171FEAFF012660C7F
:101040007DFF0DED30E70122D27075F004A424D8A5
:10105000F582E5F03400F583C082C083787DE0F648
:10106000A308E0F6A308E0F6A308E0F6D083D08258
:10107000120FD1787D8683088682787DB6FF0708B7
:10108000B6FF030210EAC3E58233F582E58333F548
:1010900083E58224E0F582E5833405F583787FE6F5
:1010A000704808E66044FB7402F9747DF8753001FD
:1010B000858331858232120A2D120FD2A3A3787D47
:1010C000E60856B4FF030210EA787D86F053F07FFD
:1010D00008E6C39EC0E0E5F09FD0F0400445F07004
:1010E00009787DE6A2E79270DBBD120FD3BD003D0B
:1010F000B2701231F34033203130201B0E30320BEE
:10110000204E05307024800320701FA270924E92F2
:10111000E0A24F92E1F5F013924F65F030E00B2022
:101120004F0512329A80031232A9021042ED14C008
:10113000E0030303540F247DF8D0E0540704FB744C
:1011400000D333DBFD307005FBE24B8004F4FBE29F
:101150005BF2021042120A52120A83120A52120A57
:101160008AD2E0120A52120A8F120A5222120A7806
:10117000C2937454121155E4120A52120A65F60809
:10118000D9F9D29322120A78C2937484121155E6C7
:10119000120A5208D9F9D2932290FC0075300475D6
:1011A0003100753200C082C083754CFA12093712C3
:1011B0000AA885306E85316D7908787D120937125D
:1011C000116D121395D083D0827044C082C0837891
:1011D0008186830886821212464024787F8683089F
:1011E00086821212464018121265E582600AE56B8B
:1011F000B56D0CE56CB56E07D083D08202122178F4
:101200007FE6249AF61213D8126164D083D0820547
:1012100031E53170020530A3E582458370871212F3
:10122000287533FF7534FF22787F760008760078C2
:10123000817600087600087600087600756E0475E1
:101240006D001213B422C082C083E5822400F582AF
:10125000E5833480F5834005D083D08222D083D0CB
:101260008290000022E58275F008A4F582E5F0C5C1
:101270008375F008A42583F583E5F03404F56CE567
:10128000822400F582E5833400F5835002056C85E5
:10129000836B22126174D083D08222C082C08312F9
:1012A000136E70EF787F868308868212124640E3C1
:1012B00012126512164F787D76007881E518F608CF
:1012C000E519F60876000876007408F9747DF8854B
:1012D0006C308583318582321209827404F97481FD
:1012E000F8856C30858331858232120A2D75F004C1
:1012F000787D7981E667600280990809D5F0F5125A
:101300001375787F8683088682A3121246787FA69B
:101310008308A68278818683088682121246787FA7
:10132000E66583700A08E665827004A312124678A7
:1013300081A68308A682C06EC06D856C6E856B6DBC
:101340001213B4D0E0D0F0B56D09C5F0B56E0280CF
:1013500018C5F0C06EC06D85F06EF56D787FE6241F
:1013600099F61213D8D06DD06ED083D0822212138A
:101370007512139522856E30856D31753200120914
:1013800037120AA87908787D12093712116D853055
:1013900033853134227882E6182618261826182438
:1013A0005566700F7882E618661866186618661813
:1013B000649966221213BB1213D8227882E618268B
:1013C00018261826182455F67882E6186618661826
:1013D000661866186499F622856E30856D3175320F
:1013E00000120937120AA81209377908787D1211FC
:1013F00085120937120B6E120937120AB585303380
:101400008531342212136E7030787FE6C0E008E632
:10141000C0E0088683088682C3D0E09582F582D03A
:10142000E09583F58350104582600CE5822400F539
:1014300082E5833480F583C322900000D322C2B6B4
:10144000121404E433C0E075380074031250B9E597
:101450001E1250B9E51F1250B974531250B9D0E0A2
:101460001250B974001250B974001250B9E58312C9
:1014700050B9E5821250B9E5381250B93099FD22C1
:10148000C2B6E5366004F4FF8004FF1212287538F6
:101490000074031250B9E51E1250B9E51F1250B97D
:1014A00074561250B9EF1250B9E5381250B930994C
:1014B000FD227401C0E0787D75F008E4F608D5F0EF
:1014C000FBD0E0D32212140440E860E878818683E0
:1014D0000886821214D8C322C082C083E58275F0C8
:1014E00008A4F582E5F0C58375F008A42583F5838B
:1014F000E5F03404F56CE5822400F582E5833400E0
:10150000F5835002056C7408F9747DF8856C30859C
:101510008331858232120A2DD083D08222121404A4
:101520007F0850051212287F00787F865B08865C52
:1015300008865D08865EC2B675380074031250B91D
:10154000E51E1250B9E51F1250B974541250B9E596
:10155000361250B9EF1250B9E536603CE55E655C75
:10156000F5F0E55D655B45F0600B855E82855D832A
:101570001214D880031214B4855E82855D83A31291
:10158000124685825E85835D787D75F008E612508F
:10159000B908D5F0F8D536C4E5381250B93099FD00
:1015A000C322E5367007C2AF1214045005E536F4C5
:1015B000800C7881A65D08A65E1213B4E536D2AF22
:1015C000C0E0C2B675380074031250B9E51E12505F
:1015D000B9E51F1250B974551250B9D0E01250B984
:1015E000E5381250B93099FDD322C2B6753800746F
:1015F000031250B9E51E1250B9E51F1250B97458C4
:101600001250B97420232354FC041250B9742012D0
:1016100050B990DB007F207404F9747DF8753001B7
:10162000858331858232120A2D787DE61250B90801
:10163000E61250B908E61250B908E61250B908A3EC
:10164000A3A3A3DFD2E5381250B93099FDD32212FB
:1016500001627883E630E402240A540FC4F97882E8
:10166000E6C4540375F00AA4F5F0E6540F25F0C360
:101670001349787EF67882E692E754C0F97880E6DE
:10168000C4540775F00AA4F5F0E6540F25F049F9A3
:101690007881E6C4540375F00AA4F5F0E6540F25EA
:1016A000F0F5F0787FE654702345F07880F6787F87
:1016B000E9F622C082C083E5301261B6E5311261DD
:1016C000B6787FE61261B608E61261B608E61261E6
:1016D000B608E61261B6120FB6D083D08222535AF2
:1016E0000F53590F5318F053190FC2AFE559232464
:1016F000AEF8E5184519F608A61A055953590FE52D
:1017000059B55A05055A535A0FD2AFC3E559955AE0
:101710005002241024F4500375640022E55AB55990
:10172000057400780022C33324AEF8E6C0E008E672
:10173000F8D0E022AC803050068C804380EF2275D8
:10174000801F00000000E58075807F540FB40F03F8
:10175000021783E5807580BF30E03230E13E30E231
:101760004A30E356E5807580DF30E02630E13230E4
:10177000E23E30E313E58030E01D30E12930E23510
:1017800030E33C74FF0217CC74000217CC740102E2
:1017900017CC74020217CC74030217CC740402171E
:1017A000CC74050217CC74060217CC74070217CC50
:1017B00074080217CC74090217CC740A0217CC748F
:1017C0000B0217CCF53E753F01021739B53EF5D532
:1017D0003FF7B4FF03021739D250F540021739C260
:1017E00090C2AFA284D284C0D0C284D290C290A250
:1017F00095B39201D290C290A295B39202D290C2B8
:1018000090A295B39203D290C290A295B39205D2C2
:1018100090C290A295B39204D0D09284D2AFD290CD
:10182000223050FDC2A075F006120702D2A075F05A
:1018300014120702E540C25022301A03754BF01211
:10184000269D205007740F301A0580F312182122AC
:10185000C22BA22BB392A722D22BA22BB392A722E8
:10186000B22BA22BB392A722F5F00303543FB4028C
:101870005BE53964086005E539B40D4DE5F089F0A4
:10188000C0F0300D1CC0E078CCE26013C3335005CB
:10189000D0E00218B012062750F6D0E00218A1D00E
:1018A000E0D0F0A9F05403B4020D1218500219361A
:1018B000D0F0A9F0021936B40106121858021936F0
:1018C000B40306121860021936021934B40365E530
:1018D0003A64086005E53AB40DEFE5F089F0C0F030
:1018E000300D1CC0E078CDE26013C3335005D0E06A
:1018F00002191212062750F6D0E00218FFD0E0D0ED
:10190000F0A9F05403B40211C22CA22CB392A60287
:101910001936D0F0A9F0021936B4010AD22CA22C43
:10192000B392A6021936B40309B22CA22CB392A624
:1019300080048000D322C322797D776BE4A24F928A
:10194000E0A26992E1A26A92E2A22A92E3A24E92F6
:10195000E4A26B92E5A26C92E709F7097700097798
:101960000009A73909A73A09A73B0977007408F9C4
:10197000747DF875300275318E75320012098274EB
:1019800010F9747DF875300275318E7532081209C0
:101990005122D24ED24FC225C22BA22BB392A7C244
:1019A00026C22CA22CB392A6227408F9747DF87575
:1019B000300275318E753200120A2D787DB66BD2E9
:1019C000787EE6A2E0924FA2E4924E7881863908B2
:1019D000863A08863BE5397008A24FB3922BB39242
:1019E000A7E53A7008A24FB3922CB392A67410F9EF
:1019F000747DF875300275318E753208120A0878D8
:101A00007D76FF7401F9747DF875300275318E753D
:101A100032001209822278C875F010E4F208D5F07D
:101A2000FB74FF78D0F278D1F222D24E6F20657825
:101A300074656E64656420202020202020200075BD
:101A400065FF121A16C20DC20C120F247061120922
:101A5000B37401F97465F87530017531037532A0FE
:101A6000120A2D7410F974C8F875300175310375B8
:101A700032A1120A087410F9748DF87530017531AD
:101A8000037532C0120A087410F9749DF87530019C
:101A90007531037532D0120A087402F97471F87541
:101AA00030017531CE753200120A08D20DD20C22E7
:101AB00022E8C0E0786DE2F573D0E0F822E8C0E0FB
:101AC000786EE2F573D0E0F822E8C0E0786FE2F5D6
:101AD00073D0E0F82275F00384B40104741A8017FF
:101AE000B4020474228010B40304742A8009B4047C
:101AF0000474428002741A227403F9746AF875300F
:101B00000075318C7532E5120A08786AE2121AD52E
:101B1000786DF2786BE2121AD5786EF2786CE21278
:101B20001AD5786FF2786AE224FD92067401F9748E
:101B300069F875300075318C7532E2120A0822742A
:101B400003F9746AF875300075318C7532E5120945
:101B5000517401F97469F875300075318C7532E291
:101B600012095122797D774709774D09777D0977E9
:101B7000A07404F9747DF875300075318D753220CC
:101B80001209827404F9747DF875300275318D750F
:101B90003220120982227404F9747DF875300075C0
:101BA000318D753220120A2D797FE7647D22E4A2FF
:101BB0002092E0A22192E1A22292E2797DF77401C3
:101BC000F9747DF875300075318C7532E812098230
:101BD000227401F9747DF875300075318C7532E826
:101BE000120A2D797DE7A2E09220A2E19221A2E2E1
:101BF000922222797DE4A22D92E0A22E92E1A22FE0
:101C000092E2A21892E392E492E5A23192E6A23225
:101C100092E7F709E4A23092E0A23392E1A2349273
:101C2000E2A23592E3A23792E4A23792E5A238927B
:101C3000E6A23992E7F709E4A23A92E0A23B92E1E8
:101C4000A23C92E2A23D92E3A23E92E4A23F92E540
:101C5000A24092E7F709E4A24192E0A24292E3A2F5
:101C60004492E4A24592E5A24692E6A24392E7F7A7
:101C70007404F9747DF875300075318C7532EC128E
:101C80000982797DE4A24792E1A24892E2A24992B8
:101C9000E3A24A92E4F4F709E4F4F709E4F4F774F0
:101CA00003F9747DF875300075318C7532E91209CD
:101CB00082227404F9747DF875300075318C7532A8
:101CC000EC120A2D797DE7A2E0922DA2E1922EA2DC
:101CD000E2922FA2E39218A2E69231A2E792320991
:101CE000E7A2E09230A2E19233A2E29234A2E39220
:101CF00035A2E4A2E59237A2E69238A2E79239092A
:101D0000E7A2E0923AA2E1923BA2E2923CA2E392E5
:101D10003DA2E4923EA2E5923FA2E6A2E7924009EC
:101D2000E7A2E09241A2E39242A2E49244A2E592A9
:101D300045A2E69246A2E792437403F9747DF875D2
:101D4000300075318C7532E9120A2D797DE7F4A2E5
:101D5000E19247A2E29248A2E39249A2E4924A09A0
:101D6000E7F409E7F422797DF77401F9747DF875D9
:101D7000300075318C7532E4120982227401F974D5
:101D80007DF875300075318C7532E4120A2D797D3D
:101D9000E7227401F9745BF875300075318C753287
:101DA000FC120951227401F9745BF8753000753129
:101DB0008C7532FC120A0822785BE27006785CF2BD
:101DC00008F222C2F0303E0475F03CA4AAF075F08F
:101DD00008A4FBACF0EA75F008A42CFAC374FD9BD0
:101DE000FB74FF9A785CF2EB08F2227401F9745EDE
:101DF000F875300075318D75320012095122740169
:101E0000F9745EF875300075318D753200120A086C
:101E1000227402F97473F875300075318C7532FDD7
:101E2000120A087402F97475F875300075318D75F1
:101E30003201120A08227402F97473F875300075C1
:101E4000318C7532FD1209517402F97475F87530D0
:101E50000075318D753201120951227401F97461D6
:101E6000F875300075318C7532F01209517401F932
:101E70007462F875300075318C7532F41209517442
:101E800001F97463F875300075318C7532F61209FA
:101E900051227401F97461F875300075318C753216
:101EA000F0120A087401F97462F875300075318C0B
:101EB0007532F4120A087401F97463F8753000750C
:101EC000318C7532F6120A087401F97464F87530B1
:101ED0000075318C7532F2120A08227401F97439D6
:101EE000F875300075318C7532F81209827401F979
:101EF000743AF875300075318C7532FA12098274B3
:101F000001F9743BF875300075318C7532FB12099C
:101F100082227401F97439F875300075318C75328C
:101F2000F8120A2D7401F9743AF875300075318C85
:101F30007532FA120A2D7401F9743BF87530007588
:101F4000318C7532FB120A2D227402F9741EF87559
:101F5000300075318C7532E0120982227402F974F6
:101F60001EF875300075318C7532E0120A2D22C0D2
:101F700082C083E58275F008A42420F58250020512
:101F8000F0A8F0E58375F008A4282400F583787D97
:101F900076FF7401F9747DF8753000858331858290
:101FA00032120982A3A3A3A3A37401F9747DF87567
:101FB0003000858331858232120982D083D082C27B
:101FC0000C220809E7C4F5F066540F700D08E7F518
:101FD000F066540F7004DAEAE422E6540FC5F054B8
:101FE0000FC395F0920B740122788279277A03E669
:101FF000C4540FF309E6540FF30908DAF27927788D
:10200000A17A06E6540FF6E36670080908DAF4E4EC
:10201000C25522792C78A67A06C3E3961918DAFA03
:10202000920B792C78A67A06E3540FB40F08E65485
:102030000FB40F108008E6540FB40F0B8006181968
:10204000DAE680CB740122C3E396B409028012144D
:10205000600FC3E3F5F0E695F0B409028003147055
:10206000E3E9B42704E4D255221918E366540F605B
:10207000F080D1121FE9701A3055172030157518ED
:102080005085831985821A1216DE754AB4D251D250
:1020900054E42204227408F9747DF8753000753117
:1020A0008C7532C0120A2D749FC395729572F8C355
:1020B00074829572F9AA72121FC4227408F9747D91
:1020C000F875300075318C7532C0120A2D122073EC
:1020D000227405F9747DF875300075318C7532C045
:1020E000120982227403F97482F875300075318CFC
:1020F0007532C512098222C082C083E5822420F590
:1021000082E583347DF5837401F9743CF875300001
:10211000858331858232120A2DD083D082C082C05D
:1021200083E58275F008A42420F582500205F0A80A
:10213000F0E58375F008A4282400F5837408F97489
:102140007DF8753000858331858232120A2DD08367
:10215000D082124C4322C082C083E58275F008A46D
:102160002420F582500205F0A8F0E58375F008A45C
:10217000282400F5837408F97495F8753000858378
:1021800031858232120A2DD083D08222C082C08350
:10219000E58275F008A42420F582500205F0A8F02D
:1021A000E58375F008A4282400F5837406F9747D8E
:1021B000F8753000858331858232120A2DD083D0A4
:1021C00082227405F9747DF875300075310075321E
:1021D00020120A2D749FC395729572F8C37482956C
:1021E00072F9AA72121FC422751B20751C00900080
:1021F000007405F9747DF8753000851C31851B323B
:10220000120A2D749FC395729572F8C374829572E9
:10221000F9AA72121FC46018E51B2408F51B5002AE
:10222000051CA3E583B40FC9E582B4A0C4740122E0
:102230001220F7E422200C0280AE751B00751C00F2
:1022400075699F756A0FE569251BC2E0F582E56A2D
:10225000351CF583C082C083E5822400F582E583C6
:10226000341BF5837402F9747DF875300185833170
:10227000858232120A2D787D86830886821220F7A5
:10228000749FC395729572F8C374829572F9AA729D
:10229000121FC47005D0F0D0F022D083D082C3E5E5
:1022A0008313F583E58213F582200B14E5824583C1
:1022B0006023E58224FFF569E58334FFF56A800732
:1022C000A385821B85831CC3E569951BE56A951C64
:1022D0004003022246740122300D24789579AD75B1
:1022E000F00AE3B4FF028017B43C0F0809D5F0F2FE
:1022F000900FE878D6E2F53CE42266540F60EC7467
:102300000122751B25751C009000007403F974826E
:10231000F8753000851C31851B32120A2D1220738E
:102320006018E51B2408F51B5002051CA3E583B4C7
:102330000FD9E582B4A0D47401221220F7E42278E8
:10234000A1E6540FB40F030223D9200C0280B37509
:102350001B00751C0075699F756A0FE569251BC216
:10236000E0F582E56A351CF583C082C083E58224EE
:1023700000F582E583343BF5837402F9747DF875CA
:102380003001858331858232120A2D787D8683085B
:1023900086821220F71220737005D0F0D0F022D080
:1023A00083D082C3E58313F583E58213F582200B86
:1023B00014E58245836022E58224FFF569E58334D4
:1023C000FFF56A8007A385821B85831CC3E5699599
:1023D0001BE56A951C4002808274012278957A057B
:1023E00079A9E6540FC4F5F008E6540F45F0F70854
:1023F00009DAEF22C2A3C262C2A2C265C2A1C2644C
:10240000D2A075F0021205DBD5F0FA20A02BD21A6B
:10241000D2A3C262C2A2D265D2A1C264D2A4C26354
:10242000120675B28475F00F1205DBD5F0FA30A0F4
:10243000EF1224CAC2AF026CB7D2A0120EC0700C49
:10244000122479121B967004121A3F22C21A754C7C
:10245000FA75F0641205DBD5F0FAC2A0C2A2C2651B
:1024600075F0641205DBD5F0FAD2A0D2A2C265D213
:10247000A01205F320A0D58095121BD1121CB21218
:102480001D7CA2E0924BA2E1924CA2E2924D121D61
:10249000A5121DFE121E92121F12121E117410F9A7
:1024A00074ADF87530017531CE753220120A0812FC
:1024B0001F5C121AF8121DB822C2A3C262C2A2C2C5
:1024C00065C2A1C264D2A4C26322D21A126086403D
:1024D000E8C2A3C262C2A2C265C2A1C264D2A4C23F
:1024E00063C01EC01F787D9000007A08E6F008A344
:1024F000DAFA1225B8787D9000007A08E0F608A391
:10250000DAFA900000125DCB1220D11220E4D01F25
:10251000D01E121F49125E48121228120BB52275E6
:102520001E30751F30C220C221C222C22DC22EC24F
:102530002FC218C231C232C230D233C234C235C205
:1025400037C238C239C23AC23BC23CC23DC23EC2A7
:102550003FC240C241C242C243C244C245C246C257
:1025600047C248C249C24A78737422F2087400F222
:1025700078757406F2087400F2C24BC24CC24D78F2
:102580005B7404F2785E7409F278617401F2786227
:102590007402F278637404F278647404F275390793
:1025A000753A00753B0074017869F2786AF2E408C4
:1025B000F208F2C20DC20C22120F6512251F121F63
:1025C00049121BAE121BF3C2E0A24B92E0A24C9246
:1025D000E1A24D92E2121D66121D92121DEB121E17
:1025E0005B121EDB121E36121B3F121B641267C5E4
:1025F00022306704C267800975F00C20B305D5F05E
:10260000FAD322C322201A31E8C0E0E9C0E0EAC0D0
:10261000E02006261225F150171227D975520078AE
:102620006AE2600C75F0031205DBD5F0FA123A95F8
:10263000D0E0FAD0E0F9D0E0F8223074F3C082C0E4
:1026400083E5717008126E744003122659121AB194
:10265000126E4AD083D08280D7D26EC26F786AE27F
:10266000B40F028013B41007124E32D25D802D7564
:10267000F00384E5F0B40007124F15D25D801DB45D
:102680000107124DB1D25C8013B40210124D3C40D0
:102690000B7859E583F208E582F2D25E22D25F80A0
:1026A00008C25F122711753D00C219D267754CFA36
:1026B0007440301A02740CF549C25DC250E549609D
:1026C0003B122605205D3575F0031205DBD5F0FAC7
:1026D00012073C201A0320191A3050E1D26F205FF4
:1026E0001B754960121821B40B0D75F0081205DB3B
:1026F000D5F0FAD25D800512270480C1C25CD2AF4A
:10270000754CFA22533D07F8E53D24A1C8F6053D76
:102710002278A175F00874FFF608D5F0FB22305C32
:1027200009201F03D21F22C25C22C21F22D297128D
:102730002737C29712273722C297C2B5122737D23E
:1027400097122737D2B5122737C29712273775F05D
:10275000083392B512272DD5F0F722D2B775F008BD
:10276000D297122737A2B7C29712273733D5F0F086
:1027700022C297C2B5122737D297122737D2B51285
:102780002737C297122737D2B512272D12272D12BD
:10279000272D22D297D2B77473122738744B122781
:1027A00038745012273812060B7408122738122773
:1027B0005B23243F3013022420543F4480122738E7
:1027C000746B1227381205F3746812273812060B3F
:1027D000746012273812277122C2ABC28ED2AFD2D8
:1027E00097D2B722C2ABC28ED2AF7455122738D25D
:1027F00097D2B722C2AFC28E53890F438910758B0F
:1028000019758DFCC28FD28ED2AFC259D2BBD2AB5A
:102810003059FD22C0D0A2B79258D259D0D0C2AB05
:10282000C28EC28F758B0D758DFED28EC2AF32D225
:102830005F8004D267C25FC219754CFAD21E744021
:10284000301A02740CF549122711753D00C25DC2A1
:102850005CC250C25EC26012073C201A0320194DB0
:10286000B207300720B20830081B2012071227D900
:10287000B213D21E201A0E122605205D32205C2FC4
:10288000205E2CD21E3050347869E27004C2508031
:102890002BD26F205F197549601227D9D21E1218EA
:1028A00021B40B1575F0081205DBD5F0FAD25D12D4
:1028B00027D9754CFA12660C22122704E54960EFFD
:1028C00012660C301E0FC21E7869E270051227E4F2
:1028D0008003122793C28EC2ABD2AF20B7063060FE
:1028E000FA02285512073C30B7063060FA02285524
:1028F00079081227F43058DD208FDA20B7FAD9F2A0
:102900007895790B7B007A057C00C2571227F4205A
:102910008FC320B70520580580F52058F2A25850E3
:1029200002B257EC33FCDAE4D93120E0C303540F90
:102930006B600280A07895790A75F000E6540FF676
:10294000700205F008D9F5E5F024F850028086D22F
:102950005C757205D212D26F0228AF30570820E0A2
:10296000030228D5808A03540FF6086BFB8097C0BA
:10297000F088F0C0F0C2AF757800785CE2F54DF5F4
:10298000F008E2F54ED2AF45F0D0F0A8F0D0F070EC
:1029900009B22A202A06C20E8002D22A202A04D294
:1029A000A58003757803D267D2612230190122789D
:1029B000A1760A087603800778A1760A08760108CE
:1029C00075F06484F608E5F075F00A84F608A6F060
:1029D000753D05D219227518C0751900751A0112B6
:1029E00016DE22754800C2537518C0751900751A95
:1029F000021216DE22D251754AB475185075190F9D
:102A0000751AFF1216DE22C20F12296F203C0C75B8
:102A1000181075190F751AFF1216DE22203C0C755E
:102A2000182075190F751AFF1216DE2275186075B9
:102A3000190F751AFF1216DE2275187075190F75A9
:102A40001AFF1216DE221267C57518C075190075B7
:102A50001A0E1216DE227877F208F2123CBB7518B5
:102A6000C0751900751A501216DE30440022401A43
:102A7000306816C268206911C2AF754D00754E01ED
:102A8000D2AFC22A757800D2A5222068FCC20F12EC
:102A9000296FD26822122C364008122E924003125F
:102AA000310822122C414008122E9D40031231138E
:102AB00022301A08C37865E4F2022C4FA2013020BC
:102AC00001B37865E233F2B4FF03022AD3022C4F3C
:102AD000022D0C2023032027F7D227300D1CC0E045
:102AE00078C8E26013C3335005D0E0022D0C120603
:102AF0002750F6D0E0022AFAD0E07861E260D1B443
:102B0000012DD2101229D6302A1C203A11C2AF75DD
:102B10004D00754E08D2AFC22A757800D2A5785EF6
:102B2000E2F548022D0C2038031229F5022D0CB4D1
:102B3000021A122A95400F302E03204F09206A06F0
:102B4000122A07022CFE122A1C022D0CB40308C202
:102B50004F122A2C022D0CB40706757B01757003E9
:102B6000B4090C204F03203903022C28022D0CB489
:102B70000A02743DB40E09D3122A6E740E022C2878
:102B8000B4340874001229AB022D0CB4350874104B
:102B90001229AB022D0CB4360874111229AB022D88
:102BA0000CB4370874201229AB022D0CB4381B74F6
:102BB00001F9747DF875300075318C7532F1120AA7
:102BC0002D787DE61229AB022D0CB4391B7401F966
:102BD000747DF875300075318C7532F1120A2D78DC
:102BE0007DE61229B8022D0CB43C06122A46022CAE
:102BF000FEB43D13204F08D24F122A39022CFEC2D8
:102C00004F122A2C022CFEB43E0D304407E4122A47
:102C100056022CFE022D0CB43F0E30440874FF12F5
:102C20002A56022CFE022D0C751890751909F51AFA
:102C30001216DE022D0C7861E2B40B03A22722C328
:102C400022204F097861E2B40D03A22722C322702B
:102C5000E22023033027DCC227300D1CC0E078C8F7
:102C6000E26013C3335005D0E0022D0C120627504A
:102C7000F6D0E0022C78D0E07861E26024B401085C
:102C8000C2101229E3022D0CB40203022D0CB4036E
:102C900007D24F122A398074B40908204F523039B4
:102CA0004F8069B40A02743DB40E09C3122A6E74CF
:102CB0000E022CF0B432028053B43302804EB4348E
:102CC000028049B435028044B43602803FB43702F2
:102CD000803AB438028035B439028030B43C028086
:102CE0002BB43D028026B43E028021B43F02801CFA
:102CF0007518A0751909F51A1216DE022D0C1009A7
:102D000003022D0C1266671206AED20922301A0891
:102D1000C37866E4F2022EABA202302101B37866DA
:102D2000E233F2B4FF03022D2F022EAB022F6820F4
:102D300023032028F7D228300D1CC0E078C9E260B8
:102D400013C3335005D0E0022F6812062750F6D087
:102D5000E0022D56D0E07862E260D1B4012DD210AD
:102D60001229D6302A1C203A11C2AF754D00754E7B
:102D700008D2AFC22A757800D2A5785EE2F5480283
:102D80002F682038031229F5022F68B4021A122A7C
:102D900095400F302E03204F09206A06122A0702A1
:102DA0002F5A122A1C022F68B40308C24F122A2C71
:102DB000022F68B40706757B01757003B4090C20F7
:102DC0004F03203903022E84022F68B40A02743D97
:102DD000B40E09D3122A6E740E022E84B434087411
:102DE000001229AB022F68B4350874101229AB0207
:102DF0002F68B4360874111229AB022F68B4370853
:102E000074201229AB022F68B4381B7401F9747D49
:102E1000F875300075318C7532F5120A2D787DE623
:102E20001229AB022F68B4391B7401F9747DF8754F
:102E3000300075318C7532F5120A2D787DE6122935
:102E4000B8022F68B43C06122A46022F5AB43D132A
:102E5000204F08D24F122A39022F5AC24F122A2C61
:102E6000022F5AB43E0D304407E4122A56022F5A5C
:102E7000022F68B43F0E30440874FF122A56022F06
:102E80005A022F6875189075190AF51A1216DE0283
:102E90002F687862E2B40B03A22822C322204F09D4
:102EA0007862E2B40D03A22822C32270E220230339
:102EB0003028DCC228300D1CC0E078C9E26013C3A2
:102EC000335005D0E0022F6812062750F6D0E002FA
:102ED0002ED4D0E07862E26024B40108C210122936
:102EE000E3022F68B40203022F68B40307D24F1223
:102EF0002A398074B40908204F5230394F8069B4A0
:102F00000A02743DB40E09C3122A6E740E022F4CCD
:102F1000B432028053B43302804EB434028049B4D8
:102F200035028044B43602803FB43702803AB43868
:102F3000028035B439028030B43C02802BB43D02AB
:102F40008026B43E028021B43F02801C7518A07513
:102F5000190AF51A1216DE022F68100903022F68EB
:102F60001266671206AED209221217DF30460E2013
:102F70004703122AB1204803122D0D8006122AB1F0
:102F8000122D0D301A08C37867E4F2023121A20332
:102F9000302201B37867E233F2B4FF03022FA502B7
:102FA00031210231DE2023032029F7D229300D1CE4
:102FB000C0E078CAE26013C3335005D0E00231DECE
:102FC00012062750F6D0E0022FCCD0E07863E26002
:102FD000D1B4012DD2101229D6302A1C203A11C2A8
:102FE000AF754D00754E08D2AFC22A757800D2A5D4
:102FF000785EE2F5480231DE2038031229F502310D
:10300000DEB4021A122A95400F302E03204F0920F9
:103010006A06122A070231D0122A1C0231DEB403DA
:1030200008C24F122A2C0231DEB40706757B0175E7
:103030007003B4090C204F032039030230FA023127
:10304000DEB40A02743DB40E09D3122A6E740E0265
:1030500030FAB4340874001229AB0231DEB43508FA
:1030600074101229AB0231DEB4360874111229AB88
:103070000231DEB4370874201229AB0231DEB438D5
:103080001B7401F9747DF875300075318C7532F759
:10309000120A2D787DE61229AB0231DEB4391B7499
:1030A00001F9747DF875300075318C7532F7120AAC
:1030B0002D787DE61229B80231DEB43C06122A468C
:1030C0000231D0B43D13204F08D24F122A390231B9
:1030D000D0C24F122A2C0231D0B43E0D304407E446
:1030E000122A560231D00231DEB43F0E3044087449
:1030F000FF122A560231D00231DE75189075190C74
:10310000F51A1216DE0231DE7863E2B40B03A2294F
:1031100022C322204F097863E2B40D03A22922C3FF
:103120002270E22023033029DCC229300D1CC0E0CC
:1031300078CAE26013C3335005D0E00231DE1206D4
:103140002750F6D0E002314AD0E07863E26024B440
:103150000108C2101229E30231DEB402030231DE9B
:10316000B40307D24F122A398074B40908204F5291
:1031700030394F8069B40A02743DB40E09C3122A73
:103180006E740E0231C2B432028053B43302804EE8
:10319000B434028049B435028044B43602803FB46E
:1031A0003702803AB438028035B439028030B43CFA
:1031B00002802BB43D028026B43E028021B43F023F
:1031C000801C7518A075190CF51A1216DE0231DE76
:1031D0001009030231DE1266671206AED209C2235D
:1031E00020560122C256751840751900751A001232
:1031F00016DE22E8C0E07861E2640360187862E2DB
:10320000640360117863E26403600A7864E2640333
:103210006003C38001D3D0E0F8221206F8300D0C11
:10322000126238400390FFF112627D22C0531232C5
:103230004AD05322300D13126238400390FFF1122E
:10324000627D5005F5531262D422E5537005755323
:10325000108023B41005755311801BB411057553EC
:10326000208013B420057553FF800BB4FF05755300
:103270000080037553FF12633DE55322C24F75185A
:103280006075190F751AFA1216DE22D24F75187072
:1032900075190F751AFA1216DE22C24F751860756D
:1032A000190F751AE01216DE22D24F7518707519B3
:1032B0000F751AE01216DE22E4A22A92E0A22B92E7
:1032C000E1A22C92E2F576757705123C3174035039
:1032D00004123DB022123D8A788EE6C0E0304712DB
:1032E000D0E0C0E0540712330CD0E0C0E054071225
:1032F000330C304814D0E0C0E0C4540712355AD023
:10330000E0C0E0C4540712355AD0E022A227302092
:1033100001B34007D320E10A023559C320E203027A
:103320003559302001B3301A08C37865E4F202340D
:103330009C400602349E0235592023032027F7D2F1
:1033400027300D1CC0E078C8E26013C3335005D0AD
:10335000E002355912062750F6D0E0023360D0E083
:103360007861E260D1B4012DD2101229D6302A1C26
:10337000203A11C2AF754D00754E08D2AFC22A7502
:103380007800D2A5785EE2F548023559203803125C
:1033900029F5023559B4021A122A95400F302E032E
:1033A000204F09206A06122A0702354B122A1C02F6
:1033B0003559B40308C24F122A2C023559B40706F6
:1033C000757B01757003B4090C204F03203903028B
:1033D000348E023559B40A02743DB40E09D3122A50
:1033E0006E740E02348EB4340874001229AB0235A8
:1033F00059B4350874101229AB023559B436087423
:10340000111229AB023559B4370874201229AB02C6
:103410003559B4381B7401F9747DF8753000753175
:103420008C7532F1120A2D787DE61229AB023559DE
:10343000B4391B7401F9747DF875300075318C75E1
:1034400032F1120A2D787DE61229B8023559B43CC2
:1034500006122A4602354BB43D13204F08D24F12B4
:103460002A3902354BC24F122A2C02354BB43E0D7D
:10347000304407E4122A5602354B023559B43F0E48
:1034800030440874FF122A5602354B02355975181C
:1034900090751909F51A1216DE02355970FB2023B2
:1034A000033027F5C227300D1CC0E078C8E2601356
:1034B000C3335005D0E002355912062750F6D0E04C
:1034C0000234C5D0E07861E26024B40108C2101271
:1034D00029E3023559B40203023559B40307D24F28
:1034E000122A398074B40908204F5230394F80694C
:1034F000B40A02743DB40E09C3122A6E740E02356A
:103500003DB432028053B43302804EB43402804959
:10351000B435028044B43602803FB43702803AB4F6
:1035200038028035B439028030B43C02802BB43D7F
:10353000028026B43E028021B43F02801C7518A090
:10354000751909F51A1216DE0235591009030235EC
:10355000591266671206AED20922A228302101B3A1
:103560004007D320E10A0237A7C320E2030237A7AE
:10357000302101B3301A08C37866E4F20236EA401B
:10358000060236EC0237A72023032028F7D2283082
:103590000D1CC0E078C9E26013C3335005D0E002CF
:1035A00037A712062750F6D0E00235AED0E0786299
:1035B000E260D1B4012DD2101229D6302A1C203A53
:1035C00011C2AF754D00754E08D2AFC22A75780092
:1035D000D2A5785EE2F5480237A72038031229F514
:1035E0000237A7B4021A122A95400F302E03204F3B
:1035F00009206A06122A07023799122A1C0237A7E5
:10360000B40308C24F122A2C0237A7B40706757BF1
:1036100001757003B4090C204F032039030236DC16
:103620000237A7B40A02743DB40E09D3122A6E748D
:103630000E0236DCB4340874001229AB0237A7B48A
:10364000350874101229AB0237A7B436087411126A
:1036500029AB0237A7B4370874201229AB0237A769
:10366000B4381B7401F9747DF875300075318C75B0
:1036700032F5120A2D787DE61229AB0237A7B4394C
:103680001B7401F9747DF875300075318C7532F555
:10369000120A2D787DE61229B80237A7B43C06122B
:1036A0002A46023799B43D13204F08D24F122A39C7
:1036B000023799C24F122A2C023799B43E0D30447A
:1036C00007E4122A560237990237A7B43F0E304456
:1036D0000874FF122A560237990237A77518907599
:1036E000190AF51A1216DE0237A770FB20230330E1
:1036F00028F5C228300D1CC0E078C9E26013C3333E
:103700005005D0E00237A712062750F6D0E0023766
:1037100013D0E07862E26024B40108C2101229E3F9
:103720000237A7B402030237A7B40307D24F122A05
:10373000398074B40908204F5230394F8069B40A77
:1037400002743DB40E09C3122A6E740E02378BB494
:1037500032028053B43302804EB434028049B4350F
:10376000028044B43602803FB43702803AB4380253
:103770008035B439028030B43C02802BB43D0280E5
:1037800026B43E028021B43F02801C7518A0751932
:103790000AF51A1216DE0237A71009030237A7121C
:1037A00066671206AED209221238BA12396D221299
:1037B00038C712397A22B211300D1CC0E078CCE241
:1037C0006013C3335005D0E002383512062750F697
:1037D000D0E00237D7D0E0E539700302384324F84F
:1037E0004005E53902384EE539B40904A20E805689
:1037F000B40A04A210804FB40C03D38049B40D0B5B
:103800003025030238D4D225D3803BB40E04A20F56
:103810008034B40F08C3E57B6001D38029B4100A5B
:10382000E579457AC36001D3801CB4110512506D4F
:1038300080140238D4B40D062025030238D4C225E2
:10384000C38003A24FB3922BB392A70238D4301196
:1038500066304A03304F175351037851A2E2825128
:103860004030A2E082524012A2E182534018C22BA3
:10387000A22BB392A776000238D4B60102801D763F
:10388000017550408016B60202801176027550A074
:10389000800AB60302800576037550F0D261E550C8
:1038A00023F55020E00AC22BA22BB392A70238D4F2
:1038B000D22BA22BB392A70238D4E539B40B07D28E
:1038C0002BA22BB392A722E539B40B07C22BA22B54
:1038D000B392A722300D1CC0E078CDE26013C33351
:1038E0005005D0E002395112062750F6D0E00238D8
:1038F000F3D0E0E53A700302395F24F84005E53A79
:1039000002396AE53AB40904A20E8056B40A04A248
:1039100010804FB40C03D38049B40D0B3026030242
:103920003987D226D3803BB40E04A20F8034B40F63
:1039300008C3E57B6001D38029B4100AE579457A94
:10394000C36001D3801CB4110512506D801402397C
:1039500087B40D06202603023987C226C38003A23E
:103960004FB3922CB392A6023987023987E53AB455
:103970000B07D22CA22CB392A622E53AB40B07C2B5
:103980002CA22CB392A62222B40207205D07C25CAF
:10399000C25E023A16C082C08390EA60E53D606371
:1039A00024FB405F78A1E6540F758300F582D53D76
:1039B00002805075F00AA4F58275830008E6540F62
:1039C0002582F582D53D02803AE58275F00AA4F59C
:1039D0008285F08308E62582F58250020583D53D75
:1039E000028020E58275F00AA4F582C0F0E58375B7
:1039F000F00AA4D0F025F0F58308E62582F5825080
:103A00000205837859E583F208E582F2C25DC25C63
:103A1000D25ED083D08222C289C28BD2B4C2942219
:103A2000C0F075F0FAD5F0FD75F064D5F0FDD0F07A
:103A300022123A20123A20123A20123A20123A2048
:103A4000123A2022D2B4C29475F0051205F320B3C5
:103A5000061205F330B303D5F0F11205F322C0F0DE
:103A600075F008A2E7B39294C2B4123A20C294D27D
:103A7000B4123A20C0E0E430B301040030B30104D2
:103A80000030B30104D36003D5E001C3D0E033D5E7
:103A9000F0D1D0F022D2B4C294D2B3123A20C2B440
:103AA000123A31D2B4123A31201A03306F1C788D99
:103AB0007601087480F608A2A3B392E4F674900825
:103AC000F608F608F608F6023B0A788D76030876C3
:103AD00080087480A26292E5A2A3B392E4201A083F
:103AE000A26592E1A22A92E0F6087480201A1220C0
:103AF0006F0FE55254074480A26492E5A2A1B392ED
:103B0000E4F6087480F608F608F675F007788D7EFE
:103B1000007F00E62EFEE6123A5EF62FFF08D5F093
:103B2000F2EED333123A5EF8EFD33368707B788DC0
:103B3000B6FF760562E56224FE5014756202201C11
:103B40000ED21C7518C0751900751A031216DE20E6
:103B50001A08786AE26003306F03023C067893E645
:103B600020E36D20E25D20E13E788EE6B600380865
:103B7000B64220757B017570037518B07519007514
:103B80001A001216DE7518C0751900751A0712167C
:103B9000DE8073B6551108B6000D087959E6F308B2
:103BA00009E6F3D25ED26E805DE5626014D56211E3
:103BB000301C0EC21C7518C0751900751A04121637
:103BC000DE8043788E863D08D25D79A17A04800B31
:103BD000788ED25C75720579957A05D26E75F00F84
:103BE000E6C4540FF755F0F5F009E6540FF755F019
:103BF000F5F00908DAEAE5F0B40F051977EEC25CD2
:103C0000786AE2123988123A4422786AE224FD4046
:103C10000FE2600C75F0031205DBD5F0FA123A954D
:103C200022306E0C7518B0751900751A001216DE68
:103C300022D2B4C294D2B3123A20C2B4123A31D2D0
:103C4000B4123A31788DE577540FC44407F608E58D
:103C50007623A2E392E5A2E292E3542AD2E7F608A1
:103C6000E576A2E392E1A2E492E3542AD2E7F608D1
:103C7000E576A2E692E1A2E792E3540AD2E7F6746F
:103C80008008F608F608F675F007788D7E007F004C
:103C9000E62EFEE6123A5EF62FFF08D5F0F2EED3DE
:103CA00033123A5EF8EFD33368700B788DB6FF06A7
:103CB000123A44C38004123A44D3227577087877C5
:103CC000E2F576123C3174004005123D8A80031201
:103CD0003DB07577097878E2F576123C3174014091
:103CE00005123D8A8003123DB0227577047576FF78
:103CF000123C3174025004123DB022123D8A789079
:103D00007954E6F30809E6F3087956E6F30809E67C
:103D1000F3788EE6A2E092E25414F5F008E623A2CE
:103D2000E592E0540345F0F5F07858E265F0C0E024
:103D3000E5F0F2D0E030E21FC0E0C0F0E5F075F051
:103D40004930E20375F04A7518C075190085F01AFC
:103D50001216DED0F0D0E054037003023D89E5F086
:103D60005403B4030575F0488013B4020575F04799
:103D7000800BB4000575F04B800375F04C7518C0CE
:103D800075190085F01A1216DE22F5F0244AF8E2C1
:103D9000B40205227402F22250FA7402F2E5F02411
:103DA00032F5F07518C075190085F01A1216DE226A
:103DB000F5F0244AF8E26017D5E013F2E5F0243C70
:103DC000F5F07518C075190085F01A1216DEF2228A
:103DD000D2B4C294D2B3123A20C2B4123A31D2B49D
:103DE000123A31788DE577540FC44403F608768093
:103DF000087480A26292E5A2A3B392E4A26592E164
:103E0000A22A92E0F6087480A26492E5A2A1B3927D
:103E1000E4F6087480F608F608F675F007788D7EEB
:103E2000007F00E62EFEE6123A5EF62FFF08D5F080
:103E3000F2EED333123A5EF8EFD333687071788DB7
:103E4000B6FF6C7893E620E33020E22020E1607832
:103E50008EE6B6005A08B6551108B60052087959D0
:103E6000E6F30809E6F3D25E804A8043788E863D09
:103E700008D25D79A17A04800B788ED25C757205C8
:103E800079957A0575F00FE6C4540FF755F0F5F003
:103E900009E6540FF755F0F5F00908DAEAE5F0B451
:103EA0000F051977EEC25C7870E21239888005122E
:103EB0003A44D322123A44C322700575641E80022C
:103EC000D21522C298C29932201AF8309918C29994
:103ED000205B05753500800EC0E0C0D075D0101293
:103EE00041BCD0D0D0E020980132C298205BFAC00B
:103EF000D0C0E0E8C0E0305A05C25A754200E5463D
:103F000024FE4003754602E54220E712E5425407CD
:103F10002324B0C0E074003440C0E0E59922543F4F
:103F2000232324A3C0E07400343FC0E0E5992215A8
:103F3000630240A20240A2D563FAB54509757C012F
:103F40007542000240A80240C0B462FA0240A202D8
:103F500040A2B42AF10240A2F56324C6E56340E61C
:103F600024F5E56350E005630240A27820F2156372
:103F70000240A27821F215630240A27822F2156372
:103F80000240A27823F215630240A27824F215635E
:103F90000240A27825F215630240A27826F215634A
:103FA0000240A20240D600023F4900023F4F0002F9
:103FB0003F5200023F5800023F2F00023F2F0002F5
:103FC0003F2F00023F2F00023F6B00023F730002B1
:103FD0003F7B00023F8300023F8B00023F930002C1
:103FE0003F9B00023F3700023F3700023F3700028D
:103FF0003F3700023F3700023F3700023F370002E1
:104000003F3700023F3700023F3700023F370002D0
:104010003F3700023F3700023F3700023F370002C0
:104020003F3700023F3700023F3700023F370002B0
:104030003F3700023F3700023F3700023F370002A0
:104040003F3700023F3700023F3700023F37000290
:104050003F3700023F3700023F3700023F37000280
:104060003F3700023F3700023F3700023F37000270
:104070003F3700023F3700023F3700023F37000260
:104080003F3700023F3700023F3700023F37000250
:104090003F3700023F3700023F3700023F37000240
:1040A00040D605422545F545D0E0F8D0E0D0D032E5
:1040B000800E802A802D8030803280348040803E87
:1040C000B4090875450075420080D7B442087545AB
:1040D0000075428080CC75450075420080CAB51ECF
:1040E000DF80BFB51FDA80BAF54380B6F54480B2F1
:1040F000B545CD75462012410075420080AA80D694
:10410000854337126B34D25BE537B446030251392D
:10411000B44704126B4A22B4500E854436126B0F1A
:10412000C2ACC25B75750722B45312854436E544B0
:10413000700A126B0FC2ACC25B75750222B4540ECA
:10414000854436126B0FC2ACC25B75750122B45543
:104150000E854436126B0FC2ACC25B75750322B478
:10416000560E854436126B0FC2ACC25B75750422C5
:10417000B4570E854436126B0FC2ACC25B75750521
:1041800022B4580E854436126B0FC2ACC25B7575F3
:104190000622B44E13854436E544B4010B126B0F6E
:1041A000C2ACC25B7575092224BF24E64004854475
:1041B0003622C25B22C5382538C53822E53524F0C1
:1041C000400EE5352324DBC0E074003441C0E0221A
:1041D000759906C25B753500D2B622802F80348077
:1041E0003680388039803E804680488051804F80BC
:1041F0004D804B80468050800E024278753503F525
:10420000991241B5053522740002423175380074A7
:104210000380ECE51E80E8E51F80E40242D4E53827
:1042200075350F80DA12171C123EB9883680D0E53A
:104230003680C9E536A24F92E080C1753503A836B5
:104240000536E676FF80B8E536C313602714700B99
:10425000A22792E0B392E1440480D614700BA22806
:1042600092E0B392E1440880C8147008A22992E059
:10427000440C80BD74FC80B9E53614702574083098
:104280006812306904440680A8306A04440380A19F
:104290004407809DA26992E0A26A92E1A22A92E27A
:1042A000808F1470117410A22792E0A22892E1A2CC
:1042B0002992E20242311470097418A21C92E002A1
:1042C000423114700BA26B92E0A26C92E202423176
:1042D000E4024231E537B441067535040241FFB4CA
:1042E000422AE536600330151B53590F535A0FC24B
:1042F000AFE55AB55906D2AFD3024304055A535A13
:104300000FD2AFC375641E74420241FCB444552001
:104310000DF7E536C3137022B392661231F34040B5
:1043200020313D30320B204E05306634800320664C
:104330002FA266924F924E024360926614C0E00331
:104340000303540F247DF8D0E0540704FA7400D31B
:1043500033DAFD306605FAE24A8004F4FAE25AF6EE
:10436000E53780A5B44B0280030243F2E53654F8EA
:10437000B40812E5365407602B14604714604B14E0
:1043800060670241D0B420030241D0B42813E5365F
:10439000A2E0924F756F015003756F02E53702413D
:1043A000FC0241D0751AF4C26AC26920686BC2AFC0
:1043B000754D00754E01D2AFC22A757800D2A5D2D4
:1043C000678056751AF3D26A80DF751AF2D269C215
:1043D0006A206845C2AF754D00754E01D2AFC22A42
:1043E000757800D2A5D2678030751AF1D269C26A99
:1043F000801FB4430FB5360375470375350775360F
:10440000A90241FFB44A23E536701C206A19751AC7
:10441000F0C20F20680312296F75181075190F125A
:1044200016DEE5370241FC0241D0B445067535067B
:104430000241FFB4510675350C0241FFB44D0EE543
:1044400036121868E5375002B2E7024309B44C0649
:1044500075350E0241FFB4460280C9B4470280C4DC
:10446000B44F08C251C252C25380B90241D0E5666E
:10447000C2726002D272E553F554C254205E0C2021
:104480005C1B305D030244FA024A921206E6785938
:10449000E2F58308E2F5821220F702462D1206E6C5
:1044A0001223DC12223560081222D8703002462D09
:1044B000206E05206B0A8003206C05124B06501AF3
:1044C000C082C0831206B81226A1D083D082305D8C
:1044D0000CE53D6008122073700302462D754B3CBD
:1044E000D5471475183075190085471A1216DE75F0
:1044F0004703D252754AB4024A7D1206E6E53D6092
:10450000F6B40206125FA4024A92206E1920190323
:10451000303313B4051078A1B60A0B08B601028037
:1045200008B6030280030245C508E675F00AA40830
:104530002675F00AA40826C5F0703B78A2B60339A8
:10454000201909C0F0124AC1D0F0502A85F05385D5
:10455000F0541206AE20190F7518C0751903855353
:104560001A1216DE024A927518C075190285531A7E
:104570001216DE024A92024A75201909C0F0124A48
:10458000ADD0F050F185F05320190E7518C0751993
:104590000685531A1216DE800C7518C0751905852C
:1045A000531A1216DE1262D8124AF3D2A2C265C2A0
:1045B000A1D2641206B8122833A25C725D500302C5
:1045C000447C024A9212233F7047206E05206B0AFA
:1045D0008003206C05124B0650531206B8C082C0EF
:1045E00083122833D083D082305C23C082C08312F0
:1045F00006E61223DCD083D082749FC39572957235
:10460000F8C374829572F9AA72121FC4601F024423
:10461000DD7869206F02786AE2B40F0A124DEEC2AB
:104620005DD25C0244A0B4100280F180E1306E33B0
:10463000300D1CC0E078D4E26013C3335005D0E0E5
:1046400002466312062750F6D0E002464FD0E075CE
:104650007702786BE27870F2121ABD124F63500342
:104660000244DD306F33300D1CC0E078D5E26013BA
:10467000C3335005D0E002469912062750F6D0E029
:10468000024685D0E0757703786CE27870F2121AF2
:10469000C9124F6350030244DD126CBF4003123A4B
:1046A00017E53C0470030244DD754B00754703C2F7
:1046B00053C252205402C251C082C083124BADD0AB
:1046C00083D0825006124A2E024A92C082C08312C0
:1046D0000BCBD083D0825006124A2E024A92E5823A
:1046E00024CEE58334FF5017124AF44012C216C29A
:1046F000171231F35006124A1F024A920249391228
:104700002A955012124A1F0248D0124A190248D064
:10471000124A130248D0206AF1302E03204FF130A4
:104720006E037860E2306F02E53C600923120627D1
:10473000400302473E024785124A0D0248D0300D21
:10474000F73018F4303FF112508B4039A26E3040F0
:1047500001B35031300D1BC0E078D1E26012C33399
:104760005004D0E080D212062750F7D0E002477202
:10477000D0E0C082C0831269A0D083D082500612DC
:104780004A240248D030187212508B406D12694C86
:10479000A2E09216A2E19217A26E304001B3C0E0EF
:1047A000920A501E12506D5019303B0EE4A2169220
:1047B000E0A21792E1B402028008D0E01249FB02A5
:1047C00048D0D0E0B40005200A22802BB40122207A
:1047D0000A1A7518C0751900751A091216DE203BE1
:1047E00006124A290248D0124AA3800E126891800C
:1047F00009B402ED200ADB1268EC300D7E12508BFA
:104800004079300D1CC0E078D0E26013C33350050E
:10481000D0E002487B12062750F6D0E0024821D0B3
:10482000E0207216A26E9271858367858268124AB3
:104830009F1206C9756602024A92756600E5836595
:1048400067F5F0E582656845F07006124A33024864
:10485000D07518C0751900751A0C1216DE30710C5F
:104860007518B0751900751A001216DE124A5875BF
:10487000181085671985681A1216DE304F0EC2A30C
:10488000C262C2A2C265D2A4C263800CD2A3C262B9
:10489000C2A2C265C2A4C263A26E920FD20E124A15
:1048A0009B12296F30460620A8031232B8123C2111
:1048B000124A5875181085831985821A1216DE124D
:1048C00006AE30440BC082C083124CCED083D0825F
:1048D000124AFD5009124C4330E103024A92123150
:1048E000F340F8C2A1D264D2A4C263755200123C54
:1048F0000A1220F7C082C083122833D083D08220CE
:104900005E09205C17205D2C024A921206E6785957
:10491000E2B5831D08E2B58218024939749FC39538
:10492000729572F8C374829572F9AA72121FC460EC
:1049300008024A7D12207370F8301824E4A21692FF
:10494000E0A21792E1B4030512691B8013B40205BB
:10495000126891800BB401051268EC80031268653F
:10496000300D1CC0E078CEE26013C3335005D0E0B8
:10497000024A7D12062750F6D0E002497FD0E0308F
:104980004125E5824583601F306E037860E2306F19
:1049900002E53C60092312062740030249A10249AF
:1049A000A7124A01024A92122AA3500F124A07750F
:1049B000F01E12070212069B024A92B24F123C21CD
:1049C000304F1A75187085831985821A1216DEC247
:1049D000A3C262D2A1C264D2A4C263801875186057
:1049E00085831985821A1216DED2A3C262D2A1C2B1
:1049F00064C2A4C2631206AE024A92126602024A5E
:104A000036126602024A36126602024A36126602FE
:104A1000024A36126602024A36126602024A36120A
:104A200066028012126602800D126602800812660B
:104A30000280031266027566007567FF7568FF12D3
:104A400037A8123C2175182085831985821A121601
:104A5000DE12069B1237AF22204903206E16E55363
:104A6000046011146565600C7518C07519018553D3
:104A70001A1216DE2212660212068A8015126602C9
:104A80001237A812068A1237AF7566007567FF7570
:104A900068FFC25DC25CE554F55322126602221221
:104AA00066022212660275F032120702227408F9B9
:104AB000747DF8753001753103753298120A2D80B6
:104AC000127408F9747DF8753001753103753290F0
:104AD000120A2D7882E6085608560460141206B8A9
:104AE0001226A1305D09E53D60051220736002C306
:104AF00022D32222E582249CE58334FF22E582240E
:104B00009CE58334FF22A24CE58245836010E58258
:104B1000249CE58334FF5004A24B8002A24D22E581
:104B2000822582F582E5833583F583E5822582F54A
:104B300082E5833583F583E5822400F582E58334BD
:104B40005BF5837404F97400F87530018583318551
:104B50008232120A08227882E654C0F5837883E60E
:104B600030E402240A2323543C4583F5837882E60B
:104B7000C4540375F00AA4F5F0E6540F25F00303BE
:104B800003F5F053F0E085F08254034583F5837814
:104B900081E6C4540375F00AA4F5F0E6540F25F03D
:104BA0004582F58222C39582E5F095832212508BCF
:104BB0005003024C35124B1F7800E2B4FF03024C45
:104BC00035120162124B56787DA68308A6827800C2
:104BD000E2F58308E2F58208E2F5F008E2124BA55F
:104BE000502B7800E2F58308E2F582787D86F008A4
:104BF000E6124BA550417802E2F58308E2F582788F
:104C00007D86F008E6124BA5402D024C357800E277
:104C1000F58308E2F582787D86F008E6124BA54020
:104C2000167802E2F58308E2F582787D86F008E6E0
:104C3000124BA55002C322D322785F74FFF208F210
:104C4000F5F022300DF3C082C083C3E58233F582D4
:104C5000E58333F583E5822400F582E583349AF514
:104C6000837402F9745FF87530018583318582326F
:104C7000120A08D083D082E5822418E58334FC40F0
:104C800005785F74FFF27860E2F5F018E222E582C1
:104C90002418E58334FC74FFF5F05031C082C083E2
:104CA000C3E58233F582E58333F583E5822400F59D
:104CB00082E583349AF5837402F9745FF8753001E4
:104CC000858331858232120951D083D08222E582D8
:104CD0002400F582E58334BAF5837401F9747DF814
:104CE000753001858331858232120A2D787DE66028
:104CF000422323C0E05403F5F0D0E054FC2400F537
:104D000082E5F034CAF5837404F9747DF8753001D6
:104D1000858331858232120A2D787DE60886F07807
:104D200077F208E5F0F275F0021205DBD5F0FA1221
:104D30003CBB2274FF7877F208F280EAE573B42274
:104D40000575F0048013B42A0575F006800BB44293
:104D50000575F00C800375F0027836E2540F704F41
:104D600008D5F0F7E2540F75F00AA4F582758300B8
:104D700008E2540F2582F582E58275F00AA4F582D7
:104D800085F08308E22582F58250020583E582756D
:104D9000F00AA4F582C0F0E58375F00AA4D0F025EE
:104DA000F0F58308E22582F58250020583C322D301
:104DB000227836E573B4220A757204799775F00883
:104DC0008024B42A0A757205799575F00A8017B4A3
:104DD000420C757205799575F00A783C80087572F9
:104DE00003799975F006E2F70809D5F0F92278956C
:104DF00079BD75F00AE3F60809D5F0F979C7E3F54E
:104E00007222789579BD75F00AE6F30809D5F0F9B4
:104E1000E57279C7F322124DB1749FC395729572F2
:104E2000F8C374829572F9AA72121FC422D083D07B
:104E30008222124DB1124E02122711C082C0837518
:104E40003D017836E2540F70E408E2540F70DE083A
:104E5000E2540FC4F5F008E2540F45F0F58308E280
:104E6000540FC4F5F008E2540F45F0F582C278788B
:104E7000A17900C3E5829410F582E5839427F58338
:104E800040030980EEE5822410F582E5833427F59E
:104E900083E96004D278F6087900C3E58294E8F5E6
:104EA00082E5839403F58340030980EEE58224E8DC
:104EB000F582E5833403F583E92078046004D27831
:104EC000F6087900C3E5829464F582E5839400F5E1
:104ED0008340030980EEE5822464F582E583340093
:104EE000F583E92078046004D278F608E58275F04D
:104EF0000A842078026002F608E5F0F6E82460F5FE
:104F00003DD083D0822279A177000975F00577FF23
:104F100009D5F0FA22124DB1124E02124F0675F069
:104F200008E573B4220478368013B42A04783880F4
:104F30000CB44204783E8005783675F006753D065F
:104F4000E2540F700608D5F0F7800979A1E2F7085E
:104F500009D5F0F922124F1512207322124E321287
:104F60002073227870E2700302502324FD4048C071
:104F700082C0831206B8125027D083D082205E26CA
:104F8000205D1B305C41749FC395729572F8C374A9
:104F9000829572F9AA72121FC4702C02502312203B
:104FA0007370240250237859E2B5831B08E2B5825E
:104FB0001665827012806CC082C0831206B8126FB0
:104FC00016D083D08250030250257870E2B40F0CC3
:104FD000124F55604E124E16604980EBB410071206
:104FE0004F5C603F80E175F00384E5F0B400071288
:104FF0004F5570D3802DB40107124E1670C980230F
:10500000B4021EC082C083124D3CE5828583F0D07D
:1050100083D08240B2658270AEE5F0658370A8806F
:105020000280A4C322D322754932D267306009C2FC
:1050300060C07712073CD077E549D36018C25EC2E2
:105040005DC25C1225F150E4123DD0205E06205D69
:1050500003305CD8C3C0D0A8777405B802027404CA
:10506000D0D04005123D8A8003123DB022E57A453A
:105070007960167871E2F5F008E245F0600BD378BC
:1050800072E2957A18E2957922C322E582B4E807A4
:10509000E583B40F02D322C322C5382538C5382290
:1050A000E54B24E94008D2A3C262D2A2C26530987F
:1050B000EFC298E599125099223099FDC299F5995D
:1050C00012509922C2A3C262C2A2C265C2B675388A
:1050D0000074051250B9E51E1250B9E51F1250B9FF
:1050E0002212060B12060B12060B1250C4E53712E1
:1050F00050B9E5381250B93099FD22120F240251EF
:1051000004120EC0C0E01250C4E5371250B9D0E00E
:105110001250B9E5381250B93099FD2212060B121F
:1051200050C4E5371250B9797DE71250B909DDF95D
:10513000E5381250B93099FD22751A00754B19D215
:105140001AE539600B54F87007C22BA22BB392A753
:10515000E53A600B54F87007C22CA22CB392A6D289
:10516000A0C28EC28CC2ADC2ABC2ACC2AF7581CE82
:1051700090517BC082C08375D00032D2AFD28C12E6
:105180006B0FC2ACD2991250E1B284754B19D29810
:105190000251B8B40922F5381250A0B51E2712509A
:1051A000A0B51F211250A0B4461B1250A0AF381258
:1051B00050A06F70101250E1D2B6D2A3C262D2A238
:1051C000C2651250A0B40ACBF5381250A0B51EF536
:1051D0001250A0B51FEF1250A0F537B46D03025264
:1051E00068B46E03025281B46F030252B8B4700304
:1051F000025305B47103025319B4730302532AB462
:10520000740302532CB47503025340B47603025363
:1052100058B4770302536CB47803025380B4790313
:105220000253A1B47A030253BDB46C030253D1B448
:105230006B030253F3B46A0302542EB4690302549D
:105240004AB468030254A9B467030254C1B46603A4
:105250000254DCB465030255A0B46403025D18B4C3
:105260006103025D730251B8AF381250A06F70F540
:105270001250E1D2B675F01E1205DBD5F0FA026CC1
:10528000B71250A0FD1424E0402B1250A02400FCC3
:105290007B001250A0FEAF381250A06F70178EF036
:1052A000EDF9747DF88B308C3185F032120A2D12B5
:1052B000511C754B190251B81250A0FD1454E070E6
:1052C000F41250A02400FC247140EA7B021250A08A
:1052D000FEEDFA787D1250A0F608DAF9AF381250D8
:1052E000A06F70D1C2A3C262C2A2C2658EF0EDF9F6
:1052F000747DF88B308C3185F0321209821250EABD
:10530000754B1980B0AF381250A06F70A8120CE224
:105310001250E1754B190251B8AF381250A06F709E
:1053200009125101754B190251B880891250A0FD24
:105330001424E040481250A02400FC7B0102529249
:105340001250A0FD1454E070341250A02400FC242C
:1053500025402A7B030252CDAF381250A06F701D3A
:1053600002537D1250EA754B190251B8AF381250F2
:10537000A06F70091250FB754B190251B80252B55B
:1053800079207D071250A0F309DDFCAF381250A040
:105390006F70EA1261B740E51201431250EA025100
:1053A000B8AF381250A06F70D412016212060B12FF
:1053B00050C4E5371250B912085C0251B8AF381228
:1053C00050A06F70661212281250E1754B190251ED
:1053D000B81250A0FE1250A0FD1250A0FCAF38121F
:1053E00050A06F7046120C4840411250E1754B19A5
:1053F0000251B81250A0FE1250A0FDAF381250A0BA
:105400006F7028120C1912060B12060B1250C4E50D
:10541000371250B9EE1250B9ED1250B9EC1250B922
:10542000E5381250B93099FD0251B80252B5AF3883
:105430001250A06F70F512060B12060B1250C4E545
:10544000371250B91216030251B8AF381250A06F7C
:1054500070D9120EB860027401C0E0120F1C600215
:105460007402D0F045F0700A120D2D121B64121256
:1054700028E4C0E01250C4E5371250B9D0E0C0E0D3
:105480001250B9E5381250B975F0031205DBD5F0AA
:10549000FA1250C4E5371250B9D0E01250B9E538CD
:1054A0001250B93099FD0251B81250A0FD1454E0C9
:1054B00070271250A02400FC2471401D7B00025272
:1054C000CD1250A0FD1454E0700F1250A02400FC27
:1054D000242540057B010252CD0252B5AF3812504F
:1054E000A06F70F512060B12060B1250C4E53712AE
:1054F00050B974011250B9744D1250B9747D1250E4
:10550000B974471250B974321250B974001250B9BC
:10551000748D1250B974201250B974DA1250B974E3
:10552000001250B9740F1250B974A01250B974809F
:105530001250B974001250B974001250B97420128C
:1055400050B974001250B974001250B9740012505E
:10555000B974001250B974001250B974001250B9E5
:1055600074001250B974001250B974001250B9741A
:10557000001250B974001250B974001250B974007E
:105580001250B974001250B974001250B97400125C
:1055900050B9E5381250B93099FD0251B80252B5F0
:1055A0001250A0F5831250A0F5822460E58334F0F8
:1055B00040EB1258891250A0FD1454E070DF7800BF
:1055C0001250A0F208DDF9AF381250A06F70CE1261
:1055D00050E175F0051205DBD5F0FA1250EA751AA4
:1055E00001300DB9300CB61258FD1258E31258971D
:1055F0001220F7789579007A0A75F00FE3540FF6C8
:1056000052F00809DAF643F0F0E5F0047895797D78
:105610007A05121FC4600B1256B85006751A0402A0
:10562000559D1258E31258971220F778A1790A7AFB
:105630000675F00FE3540FF652F00809DAF643F05E
:10564000F0E5F00478A179827A03121FC4600B128E
:1056500057565006751A0602559D1258E3125946C0
:10566000751A650251B8C0E07830E583F208E5822A
:10567000F2D0E022C0E07832E583F208E582F2D091
:10568000E022C0E07830E2F58308E2F582D0E02243
:10569000C0E07832E2F58308E2F582D0E022E582CC
:1056A0002400F582E583341BF58322E5822400F58E
:1056B00082E583343BF58322125897AB83AC82900A
:1056C0001B00C083790075300385833175320090EB
:1056D0000061120937120AA8120937120B0690004E
:1056E000617A80E0A3F5F0E0A36C7005E5F06B60F3
:1056F00017DAF0D0830583740024C0E58334C550E5
:10570000C17405125805D322D083EA2AF5F0E4C308
:1057100095F0F582125666789579007A0A75F00F41
:10572000E3540FF652F00809DAF643F0F0E5F0041E
:10573000600C12223A700A7406125805D322122203
:105740003AE5822582F582E5833583F58312569EFC
:10575000125674025B1D125897AB83AC82903B00CB
:10576000C083790075300385833175320090006104
:10577000120937120AA8120937120B069000617A33
:1057800080E0A3F5F0E0A36C7005E5F06B6017DA3C
:10579000F0D0830583740024C0E58334A550C17420
:1057A00005125805D322D083EA2AF5F0E4C395F018
:1057B000F58212566678A1790A7A0675F00FE354DD
:1057C0000FF652F00809DAF643F0F0E5F004601D38
:1057D00012234F701BAB83AC82125897EBB5830634
:1057E000ECB58202C3227404125805D32212234F4F
:1057F000E5822582F582E5833583F5831256AB1267
:105800005674025B1DF51A22C082C083E5831261C3
:10581000B6D083D082C082C083E5821261B6D083C5
:10582000D08222C082C0837F00E58224F0C0E0E500
:105830008334D8C0E05007D083D0820F80EBD0E013
:10584000D0E07F00E5822418C0E0E58334FCC0E0AE
:105850005007D083D0820F80EBD0E0D0E07F00E50E
:1058600082249CC0E0E58334FFC0E05007D083D0A1
:10587000820F80EBD0E0D0E0E58275F00A84C0F0C2
:10588000F5F0D0F0D083D08222C0E07834E583F206
:1058900008E582F2D0E022C0E07834E2F58308E245
:1058A000F582D0E0227882E61261B67883E6126152
:1058B000B67884E61261B678A1E61261B678A2E6FF
:1058C0001261B678A3E61261B678A4E61261B678E2
:1058D000A5E61261B678A6E61261B6120FB62212DC
:1058E0000FB62274001250B974001250B97400122D
:1058F00050B974001250B974001250B92275831B4C
:1059000075821B75F040C0F0C082C0837530018580
:105910008331753200120937120AA8D083D082C0B1
:1059200082C08375300385823175320012093712C7
:105930000B6ED083D08205830582D0F0D5F0C77579
:1059400033FF7534FF227401F97418F8753000754F
:105950003100753200120A2D7401F97419F875308E
:10596000017531D97532FF120A2DAC18125897E51E
:10597000822420F582E583347DF583C082C0837460
:1059800001F9743CF8753000858331858232120A42
:105990002DD083D0827401F97410F875300085839E
:1059A000318582321209517810E2F5F0E518253C74
:1059B000C395F0F518125897E58275F008A42420D5
:1059C000F582500205F0A8F0E58375F008A42824BC
:1059D00000F5837408F9747DF8753000858331858E
:1059E0008232120A2D787DE5187A082608DAFCF54D
:1059F00018789579007A0A75F00FE3540FF652F093
:105A00000809DAF643F0F0E5F00412610278A179B2
:105A10000A7A0675F00FE3540FF652F00809DAF629
:105A200043F0F0E5F00412610A7408F9747DF8752A
:105A30003000858331858232120982787DE5187ABB
:105A400008C39608DAFBF518125897C3E58233F5B8
:105A500082E58333F583C3E58233F582E58333F54D
:105A600083E5822400F582E583245BF583C082C050
:105A7000837404F9747DF875300185833185823231
:105A8000120A2DD083D0827404F97412F875300193
:105A9000858331858232120951787D7912E5197A30
:105AA0000426F5F0E3C5F0C395F00809DAF3F5191B
:105AB0007401F97418F875300075310075320012F0
:105AC00009827401F97419F87530017531D975328C
:105AD000FF12098275831B75821B75F040C0F0C0F0
:105AE00082C0837530038583317532001209371205
:105AF0000AA8D083D082C082C083753001858231EC
:105B0000753200120937120B6ED083D082058305DF
:105B100082D0F0D5F0C77533FF7534FF221256904E
:105B2000E5828583F0125682C39582C0E0E5F09548
:105B300083D0F045F07002C3225003025C38125645
:105B400090C0E0C3E58224FEF582E58334FFF5834F
:105B5000D0E0125674E5828583F0125682B5820732
:105B6000E5F0B58302C322125682AF83125690EF3E
:105B7000B58310AE82900034787DE0F6A308E0F69D
:105B8000025B9B7EFE8F8305837402F9747DF8753A
:105B90003003858331753200120A2D790075300388
:105BA0008F31753200900061120937120AA812096C
:105BB00037120B068F837582001256827D00E583B3
:105BC0006F7002AD82ED2461F5827583005002058D
:105BD00083C3EE9D20E05A03FCC082C083A3A3E0F0
:105BE000FAA3E0FBD083D082EAF0A3EBF0A3DCE9D8
:105BF000EE2461F58275830050020583787DE6F01E
:105C0000A308E6F079007530038F317532009000FB
:105C100061120937120B5A120937120B6E85303395
:105C2000853134125690EFB58303025D0C0F025B91
:105C30006C7408125805D322125682AF8312569004
:105C4000EFB58310AE82900034787DE0F6A308E0D3
:105C5000F6025C6C7E008F8315837402F9747DF804
:105C60007530038583317532FE120A2D7900753047
:105C7000038F31753200900061120937120AA812A1
:105C80000937120B061256827DFEE5836F7002AD56
:105C900082ED2461F58275830050020583C3ED9E79
:105CA00020E06B03FCC0E0C3E58224FEF582E583BF
:105CB00034FFF583D0E0C082C083E0FAA3E0FBA309
:105CC000EAF0A3EBF0D083D082DCDAEE2461F58237
:105CD00075830050020583787DE6F0A308E6F0792D
:105CE000007530038F317532009000611209371250
:105CF0000B5A120937120B6E853033853134125628
:105D000090EFB58303025D0C1F025C3DC322740952
:105D1000125805D3220252B51250A0F5831250A09A
:105D2000F582AF381250A06F70EBC01EC01F858384
:105D30001E85821F121F497401F9747DF8753000A9
:105D4000753100753200120A2D787DE6C3951EC3A9
:105D5000951FD01FD01E251E251FF67401F9747DD6
:105D6000F87530007531007532001209821250E169
:105D70000251B81250A0F583AF381250A06F709541
:105D800012060B12060B12060B1250C4E537125006
:105D9000B974001250B9E51A1250B974001250B912
:105DA00074001250B974001250B974001250B9E561
:105DB000381250B93099FD0251B8905DC2C082C00E
:105DC00083327581CE75D000026CB7C082C083E586
:105DD000822420F582E583347DF5837401F9743CD7
:105DE000F8753000858331858232120982D083D0E4
:105DF00082C082C083E58275F008A42420F5825019
:105E00000205F0A8F0E58375F008A4282400F583C6
:105E10007404F9747DF875300085833185823212FF
:105E20000982A3A3A3A3747D2404F5F07404F9E507
:105E3000F0F8753000858331858232120982D08373
:105E4000D082C20C124C8E22120EC0C0E07401F936
:105E5000747DF8753000753100753200120A2D78A6
:105E60007DE6D0F0C395F0F67401F9747DF87530D5
:105E70000075310075320012098222300D1CC0E01D
:105E800078CEE26013C3335005D0E0025F291206DA
:105E90002750F6D0E0025E9AD0E0124AF3D2A3C2B5
:105EA00062C2A1D264D2A4C2631206B812283320FF
:105EB0005C06205D35025F291206F81222357069F2
:105EC000124AFD4064206E05206B0A8003206C0599
:105ED000124B0650561206B81226A1305D4BE53D16
:105EE00060471220737042025F2BE53D603B120653
:105EF000F812233F7033124AFD402E206E05206BAE
:105F00000A8003206C05124B0650201206B8122896
:105F100033305C15749FC395729572F8C374829583
:105F200072F9AA72121FC46002D322304139E5828D
:105F300045836033306E037860E2306F02E53C6089
:105F400009231206274003025F4D025F671237A83C
:105F5000123C2175182085831985821A1216DE12CB
:105F6000069B1237AF80C2B24FC3123C21304F1A8A
:105F700075187085831985821A1216DEC2A3C26253
:105F8000D2A1C264D2A4C263801875186085831937
:105F900085821A1216DED2A3C262D2A1C264C2A442
:105FA000C263C32278A1E6B40A1708E6B405451215
:105FB00031F34009125E7B40041206AE2212068ABB
:105FC0002275F00AA4F5F008E625F0B46326D2A302
:105FD000C262C2A2D265C2A1D264D2A4C263C0E02E
:105FE0001206B81228339000001220F7205C092016
:105FF0005D35D0E012068A221206F8749FC39572AE
:106000009572F8C374829572F9AA72121FC470E275
:10601000304C441206B81226A1305DD61206F81292
:10602000207370CE0260571206F8E53D60C412205E
:106030007370BF304C211206B8122833305CB31293
:1060400006F8749FC395729572F8C374829572F9BD
:10605000AA72121FC4709B1206B8D0E012068A22E0
:10606000125E487518C0751900751A0A1216DE12EC
:1060700006AE22753C007860E4F2787D75F0087613
:10608000FF08D5F0FA22751E30751F30C26EC26F40
:1060900075F005C0F0D2A3C262C2A2D265D2A1C27D
:1060A00064D2A4C263126073122833D0F0205C095A
:1060B000205D06D5F0DD0260FD126122403F120630
:1060C000AE7882E6B4FF05C32275F005C0F0122851
:1060D00033D0F0205D06D5F0F30260FDE53DB4025B
:1060E0001C78A1E624F6401508E624F6400F78A1B6
:1060F000E62430F51E08E62430F51FC32212068A76
:10610000D3227895797D7A05800678A179827A0301
:10611000E608540FC4F5F0E608540F45F0F709DA25
:10612000EF22205C31305D3AE53D600624FD24FC21
:10613000403012610A1206B875F005C0F012282F1F
:10614000D0F0205C11205006D5F0F00261621218E8
:1061500021B40B0E8003126102753C007860E4F2FA
:10616000C322D32212617475F0641205DBD5F0FAF4
:1061700012065D2275F03C120702C2A075F03C12B7
:106180000702D2A075F014120702C2A075F03C12EB
:106190000702D2A075F014120702C2A075F0141203
:1061A0000702D2A075F014120702C2A075F01412F3
:1061B0000702D2A02222227825E254C07078E2752C
:1061C000F00A84C445F0787FF67824E254C0706603
:1061D000E275F00A84C445F07880F67823E254E052
:1061E0007054E275F00A84C445F07881F67822E2B2
:1061F000604454E07040E275F00A84C445F0C0E0A9
:106200007820E2030354C0D0F045F07882F678217C
:10621000E2602354F0701FE275F00A84C445F0C0B8
:10622000E07826E254F8700EE2C42354E0D0F04542
:10623000F07883F6C322D32290000075F019C0F0E5
:106240007402F9747DF875300185833185823212CC
:106250000A2D787EB6FF02800E18E553300D05B486
:10626000FF02E565666011E5822410F582500205A3
:1062700083D0F0D5F0C8C322D0F0A3D322300D4D87
:10628000E58224FFF582E58334FFF58375F019E597
:10629000822480E58334FE5005900000800AE58268
:1062A0002410F58250020583C0F07402F9747DF861
:1062B000753001858331858232120A2D787EB6FFD2
:1062C00002800518E6B55307D0F0D5F0C2C322D03E
:1062D000F0A3D32222026305E57C60F9757C0012ED
:1062E00061B740F11201430263087822E21261B5FE
:1062F0007821E21261B57823E21261B57824E212C6
:1063000061B502632C1201627882E6C45403E6543C
:106310000F7883E6C45401E6540F7881E6C4540F25
:10632000E6540F7880E6C4540FE6540F300D0A127D
:10633000623850051262D4800312633D22E553B4E3
:10634000FF0690040702637CB40006900287026394
:106350007CB4100690029002637CB41106900299FE
:1063600002637CB420069002A302637CE55375F0BF
:106370006484C0F0D0E01261B59002AC2220180114
:10638000227582051267C3600F75F0021205DBD516
:10639000F0FAD582EF1267C57475787D1207135035
:1063A00015207314D2731267C57518C0751900755E
:1063B0001A0D1216DE22C273120162203404203537
:1063C0002E227881E6543FF5F07973E365F0701C76
:1063D00009E37880667015203611D2361267C575CC
:1063E00018C0751900751A0D1216DE2230352A787C
:1063F00081E6543FF5F07975E365F0701C09E378A8
:1064000080667015203611D2361267C57518C075B2
:106410001900751A0D1216DE22C23622C2AC1217EE
:106420001C6024F518881912129B53590F535A0FE8
:10643000C2AFE55AB55906D2AFD3026445055A53E7
:106440005A0FD2AFC380D7D2AC227E007F709000AB
:106450000075F000E49325F0F5F0A3C3E5829EE516
:10646000839F40F0E5F0700122E5F0C0E0E5831283
:1064700061B6E5821261B6D0E01261B6C2ADC2ACBF
:10648000D21A12067520A0FA75F0C81205DBD5F0F5
:10649000FA30A0FD75F0C81205DBD5F0FA126B0FCB
:1064A0002275F064120B8120E51230E30F221205F1
:1064B000F3B2841205F3B284D5F0F322C2AFB284F2
:1064C0001205F3B2841205F3D5F0D9C2A075F032EB
:1064D0001264AED2A075F0321264AEC2A075F03272
:1064E0001264AED2A075F0321264AE75F0961264EA
:1064F000AE80D822300D3C7400788D1207224033D4
:106500007F087E007478787D120713CE13CE05E0E5
:10651000DFF4201B0E7400789D1207225005EE65F3
:106520005560108E558E537518C075190485531A11
:106530001216DE22C2AF75181075190FF51A121651
:10654000DED2AF22300D0C2068097401788D12075D
:10655000225001227477787D120713E492E0C0E0A4
:106560007476787D120713D0E033FE201B0E740181
:10657000789D1207225005EE655660D78E56EE20A4
:10658000E10630E0440265EB30E022A26A72695015
:10659000C2C26AC269C2AF754D00754E01D2AFC2A8
:1065A0002A757800D2A574F812653480A6D26AC222
:1065B00069C2AF754D00754E01D2AFC22A75780021
:1065C000D2A574F7126534808A206987D269C26ABD
:1065D000C2AF754D00754E01D2AFC22A757800D298
:1065E000A5D26774F6126534026553A22A82694007
:1065F000F7D269C26AC20F12296F74F512653402AC
:106600006553C082C083D083D082222222C2A0756B
:10661000F0141205DBD5F0FAD2A075F0141205DBE8
:10662000D5F0FA22C2A075F03C1205DBD5F0FAD203
:10663000A075F0141205DBD5F0FA2212660D126671
:106640000D12662412660D75F0641205DBD5F0FAA2
:106650002212662412660D12660D12660D75F06424
:106660001205DBD5F0FA22304F09C2A3C262D2A4D0
:10667000C26322D2A3C262C2A4C2632222300DFC32
:10668000A26B926D300D1CC0E078CFE26013C33373
:106690005005D0E00266B912062750F6D0E0026637
:1066A000A3D0E0D26B201B03206DD17518C07519E3
:1066B00000751A0F1216DE80C3C26B201B03306DEB
:1066C000BB7518C0751900751A101216DEA26C92EF
:1066D0006D300D1CC0E078D7E26013C3335005D095
:1066E000E002670712062750F6D0E00266F0D0E01D
:1066F000D26C201B03206D237518C0751900751A04
:10670000181216DE02671BC26C201B03306D0C755D
:1067100018C0751900751A191216DE22C2B675381E
:106720000074031250B9E51E1250B9E51F1250B99A
:10673000744E1250B974081250B974011250B974E1
:10674000061250B97854E2F5F0E5F01250B908E2BB
:10675000F5F0E5F01250B97856E2F5F0E5F0125098
:10676000B908E2F5F0E5F01250B9244AF8E2785899
:10677000E2547FF5F0784CE2C36001D3E5F092E794
:10678000F5F0E5F01250B975F000E5F01250B9E5FA
:10679000381250B93099FD2222120A78C2937454EB
:1067A000120A92E4120A52120A65F5F06448255F53
:1067B00033F55FE5F02560B2E003F560D9E9D293E7
:1067C000222222E4227583DD75F010753003858363
:1067D00031753200C083C0F0120937120E50D0F06C
:1067E000D0830583D5F0E47533FF7534FF1267C29B
:1067F000757900757A002202682AC082C08375828A
:1068000005C0821267C3D082601CC2A075F00F124F
:1068100005DBD5F0FAD2A075F0051205DBD5F0FA4C
:10682000D582DE1267C5D083D082E5822400C0E025
:10683000E58334DDF8D0E0C322C082C0837401F95F
:10684000747DF8753003858331858232120A2D7884
:106850007DB6020CE57A24FFF57AE57934FFF57907
:10686000D083D082221267FAC082C083F5828883E7
:10687000126839787D76007401F9747DF8753003FB
:10688000858331858232120982D083D0821267C219
:10689000221267FAC082C083F5828883C082C083D7
:1068A0007401F9747DF87530038583318582321265
:1068B0000A2D787DB60209D083D082D083D082227F
:1068C000E57A2401F57A50020579D083D082787D6B
:1068D00076027401F9747DF8753003858331858201
:1068E00032120982D083D0821267C2221267FA1252
:1068F00067FAC082C083F5828883126839787D7612
:10690000017401F9747DF875300385833185823215
:10691000120982D083D0821267C2221267FAC08223
:10692000C083F5828883126839787D76037401F913
:10693000747DF8753003858331858232120982D0E7
:1069400083D0821267C2221267F780031267FAC0EF
:1069500082C083F58288837401F9747DF8753003F1
:10696000858331858232120A2D787DE6B40102805A
:106970000CB402028007B4030280027400D083D0FA
:106980008222120A78C2937454120A92E4120A52B2
:10699000120A65B40205755F018002D9F3D2932211
:1069A000755F007583DD75F00F7530038583317574
:1069B0003200C083C0F0120937120AA812093779D1
:1069C00000126982D0F0D0830583E55F7026D5F090
:1069D000D8753003858331753200120937120AA841
:1069E00012093779A01269827533FF7534FFE55FAC
:1069F0007002D322C322C28C758A45758C5DD28CFD
:106A0000B20020000132C0D0C0E0C0F075D008D282
:106A100060121734126AF0051DE51D20E00C20E11C
:106A200009301A16E51D541F6034201A04E54C6025
:106A300002B284D0F0D0E0D0D032206505A22AB3D3
:106A400092A2E51D30E2031237B6E51D541F701106
:106A5000D261B5484DB54A5CB56464B57065B54B57
:106A60006AE4B54C4BB54972B54673B54F77B57806
:106A700078E54E454D6029E54E2401F54E5002055E
:106A80004D454D701BC20E206816206913C2AF75AC
:106A90004D00754E01D2AFC22A757800D2A5D267DB
:106AA0008088D548B0C20E754AB4D253D25680A55C
:106AB000154C80B1D54AA1C251C252C2538099151A
:106AC000648098D57098757B008093D54B937547FB
:106AD00003301A03025DBA026A581549808AD54606
:106AE0008AD25A8086154F8085D57885C2A5808147
:106AF000E51DA2E330620292A330650292A23064E7
:106B00000292A122C2B6205B02D2B6126B0F32757E
:106B1000C800C2ADC2AC75CBFF75CA9875CDFF7504
:106B2000CC98759853C298C299D2ACC2BC75C8347F
:106B30007599062275C800C2ACC2AD75980075CCB7
:106B40002B75CDEBD2AD75C8042275C800C2ACC29E
:106B5000AD759800E58A242BF5CC540F658C24EB99
:106B6000F5CDD2AD75C80422C2A8C2AAC289C28B13
:106B7000C2ACC2A9C2AB758F01120B8ED21AD2A0C1
:106B8000C2AF754D00754E01D2AFC22A757800D2E2
:106B9000A5E4F53C7860F2787D75F010F2D5F0FC54
:106BA000C268C269C26AC26BC26C753E0F75400F83
:106BB000751D04C250C251C252C253754A01754B71
:106BC00000C256D260757500C236C21CC21DD25AB0
:106BD000C25B754610E4F542F543F544F535F537EB
:106BE00012251F751E00751F80E4F548F551F550FC
:106BF000F559F55AF53FC227C228C229743778657E
:106C0000F27866F27867F2D2237547037549017806
:106C1000A97A0576FF08DAFB757C007820E47A070C
:106C2000F208DAFCC2147553FF855355C215C20D24
:106C3000C20CC23775641E756600C272C212C213DE
:106C4000C20EC20FC210C26EC26F756200756100C3
:106C500075F00A784AE4F208D5F0FB7954E4F309B8
:106C6000F37956F309F37858E4F2121A16754CFAD0
:106C7000B2847533FF7534FFD273756F00782F744B
:106C80000AF2D209757B0075700175731AC2067518
:106C90007800757900757A00758901758A3E758C62
:106CA0005DC2B9D2A9D28CD2B6126B0FD2AFD2B418
:106CB000C294D2B3B28422C2AF12193802000020AB
:106CC0000602C322121AB1126E4AD322C2AF754C09
:106CD000FAB2841205F3B2841205F3B284D2A0751D
:106CE00081CE75D000126B6812660212644A126778
:106CF000C51223F4754CFA121199126CBF75520328
:106D0000123C0A1206C2751880751903751A7D1295
:106D100016DED21B300D0F1210311264F4126544CE
:106D200012637D12667DD2A0D2AFC21AC21B0000D0
:106D30000020A0091205F320A00302240E300D1537
:106D4000303703121031300D0C1264F41265441206
:106D5000637D12667DE5666003D5660B30450312E0
:106D60003CEA1262D8800CD2A3C262C2A1D264D221
:106D7000A4C263E564700630370312641CC265D296
:106D8000A1C264126667C26EC26FD267786BE2609E
:106D90000D24FD4009757702123DD0126CBF786C4E
:106DA000E2600D24FD4009757703123DD0126CBFDF
:106DB00030460620A8031232B8122833205D08207E
:106DC0005C05205E02801A302F09305206126602DE
:106DD000026DD912446E126CBF782FE215E0F2708A
:106DE00008782F7414F2026D26026D46002074217B
:106DF000C0D0C0E0E8C0E0C0F0E54F70038573711B
:106E0000754F08C277126EC0D0F0D0E0F8D0E0D055
:106E1000D0C28932207421C0D0C0E0E8C0E0C0F008
:106E2000E54F7003857371754F08D277126EC0D02D
:106E3000F0D0E0F8D0E0D0D0C28B32C2A8C2AAC253
:106E4000B4C294C0E01205DBD0E0C2B4C294C289DF
:106E5000C28BD2B2D2B3C274754F00857371C2B8FF
:106E6000D288D2A8C2BAD28AD2AA22C2A8C2AAC240
:106E700089C28B22E573141475F00884F5F0C0F014
:106E80007836E230E002B27530E102B27530E202EB
:106E9000B27530E302B27508D5F0E7D0F0E230E029
:106EA00002B27630E102B27630E202B27630E3022C
:106EB000B27608D5F0E7207505307602C322D322DA
:106EC000E571B57307A2779275026F0AB40107A244
:106ED000779276026F0AC3E573149571403275F0AC
:106EE00004842436F8E205F0D5F006A27792E38018
:106EF00016D5F006A27792E2800DD5F006A2779221
:106F0000E18004A27792E0540FF2D57102D274228C
:106F1000857371D27422754932126E3B306005C29E
:106F20006012073CE54960113074F1E571700A1296
:106F30006E6B126E744002C322126E6BD32200007D
:106F40000000000000000000000000000000000041
:106F50000000000000000000000000000000000031
:106F60000000000000000000000000000000000021
:106F70000000000000000000000000000000000011
:106F80000000000000000000000000000000000001
:106F900000000000000000000000000000000000F1
:106FA00000000000000000000000000000000000E1
:106FB00000000000000000000000000000000000D1
:106FC000000000000000000000000000000050521F
:106FD000333032207665722E3132352E32204864BD
:106FE000773A472034303030752031342D31312D0F
:106FF00030342031323A343920204352433D00BBF3
:00000001FF
:0300000306028072
